:020000040007F3
:1020000080930020D9230700E1230700E323070082
:10201000E5230700E7230700E9230700000000008D
:10202000000000000000000000000000C5230700C1
:10203000ED23070000000000EF230700F123070055
:10204000F3230700F3230700F3230700F32307001C
:10205000F3230700F3230700F3230700F32307000C
:10206000F3230700F3230700F3230700F3230700FC
:10207000F3230700F3230700F3230700F3230700EC
:1020800099360700F3230700F3230700F323070023
:10209000F3230700F323070061350700F32307004C
:1020A000F3230700F3230700F3230700F3230700BC
:1020B000F3230700F32307000000000000000000E6
:1020C000F3230700F3230700F3230700F32307009C
:1020D0005D340700F3230700F3230700F323070011
:1020E000F3230700000000000000000000000000D3
:1020F00000000000F323070000000000F3230700A6
:1021000000000000000000000000000000000000CF
:1021100000000000000000000000000000000000BF
:1021200000000000000000000000000000000000AF
:10213000000000000000000000000000000000009F
:10214000000000000000000000000000000000008F
:10215000000000000000000000000000000000007F
:10216000000000000000000000000000000000006F
:10217000000000000000000000000000000000005F
:10218000000000000000000000000000000000004F
:10219000000000000000000000000000000000003F
:1021A000000000000000000000000000000000002F
:1021B000000000000000000000000000000000001F
:1021C000000000000000000000000000000000000F
:1021D00000000000000000000000000000000000FF
:1021E00000000000000000000000000000000000EF
:1021F00000000000000000000000000000000000DF
:10220000DFF810D000F050F900480047A55807004B
:10221000AFF300808093002030B450E8012F93B2D8
:10222000C48923448489A34228BF1B1B0489A34279
:1022300002BFBFF32F8F002007E0C3EA020340E88C
:102240000134002CE9D14FF001000A6030BC704726
:1022500050E8012FC2EA024240E801210029F7D1EB
:10226000704730B450E8022F1FFAA2F3C488A3428B
:1022700002BFBFF32F8F00200DE0C489234484895F
:10228000A34228BF1B1BC2EA034340E80234002CD0
:10229000E8D14FF001000A6030BC704750E8022FCF
:1022A000C2EA224240E802210029F7D170470346E2
:1022B00053E8022FD988B2EB324F4FF0000017BF1E
:1022C00092B241EA014142EA014104E05A68B2EBAC
:1022D000324F08BF012043E80212002AE8D17047BC
:1022E00030B4044654E8000F0D4644E80053002B78
:1022F000F8D1156030BC704730B4044654E8000F84
:1023000040EA010544E80053002BF7D1156030BCCA
:10231000704730B4044654E8000F00EA010544E871
:102320000053002BF7D1156030BC704730B4044621
:1023300054E8000F80EA010544E80053002BF7D170
:10234000156030BC704730B4044654E8000F00EB11
:10235000010544E80053002BF7D1156030BC7047ED
:1023600030B4044654E8000FA0EB010544E80053E4
:10237000002BF7D1156030BC704770B404464FF0A5
:10238000000054E8006F0D68AE4207BF44E8002328
:10239000012044E800630E60002B1CBF0020F0E722
:1023A00070BC704730B4044654E8000F88422CBF1C
:1023B000451A054644E80053002BF5D1156030BCA2
:1023C000704700001EF0040F0CBFEFF30880EFF31E
:1023D000098007F0F7B80000064880470648004724
:1023E000FEE7FEE7FEE7FEE7FEE7FEE7FEE7FEE7C5
:1023F000FEE7FEE76535070001220700202A04DB1F
:10240000203A00FA02F1002070479140C2F1200307
:1024100020FA03F3194390407047000000487047CA
:1024200000C8070040EA01039B0703D009E008C980
:10243000121F08C0042AFAD203E011F8013B00F889
:10244000013B521EF9D27047D2B201E000F8012BD5
:10245000491EFBD270470022F6E710B513460A4624
:1024600004461946FFF7F0FF204610BD421C10F845
:10247000011B0029FBD1801A704730B504460020AB
:10248000034600E05B1C934203D2E05CCD5C401B42
:10249000F8D030BD034611F8012B00F8012B002ABB
:1024A000F9D1184670470000064C074D06E0E06879
:1024B00040F0010394E8070098471034AC42F6D38B
:1024C000FFF7A2FE00D8070020D807002DE9F0434F
:1024D0008BB01446129D15F9046B00961F4680467A
:1024E00089462B460246214602A800F086FC02A936
:1024F000129A084600F07DFC129B02AA4146404613
:1025000000F067FC129B02AA2146204600F061FC05
:102510002B464A4639463846009600F06EFC129A21
:10252000394602A800F065FC02A92B46424608463F
:10253000009600F062FC02A92B462246084600964F
:1025400000F05BFC2B46424621462046009600F0F8
:1025500054FC129B22464946484600F03AFC2B4662
:1025600002AA41462046009600F047FC129B2246F4
:102570003946384600F02DFC2B464A463946384647
:10258000009600F03AFC324602A9204600F0FCFD1D
:102590000BB0BDE8F083F0B5154689B01C46074680
:1025A0000E461A462946684600F023FC23466A4632
:1025B0003946384600F00DFC23462A4669466846EF
:1025C00000F007FC23466A463146304600F001FC25
:1025D00009B0F0BD8B1802448B4200D1704713F84C
:1025E000010D02F8010DF7E72DE9F047B3F90240BC
:1025F00088461E4604F11F012023073491FBF3F7A0
:1026000008234FFA87F994FBF3F4944228BF144649
:102610004946054600F072FA22464146FFF7DAFFC6
:10262000B6F90230E4009C421FD9E41A05EB870199
:102630000022C4F120078D420ED324364A46294693
:10264000304600F066FA01280FD04B463246284645
:10265000BDE8F04700F0A4BD51F8040D20FA04F3E2
:1026600013430B6000FA07F2E5E7BDE8F0872DE9B8
:10267000F04793F9006092B004468946104631460F
:102680001546984600F05AFA002840F091804246DC
:10269000494602A800F0ADFB434602AA21460AA81B
:1026A00000F097FB02A90846424600F0A2FB434611
:1026B0002A464946484600F08CFB08F1040742468A
:1026C0002946284600F095FB3B462A4621462046EF
:1026D000009600F042FA3B462A46294628460096D4
:1026E00000F03BFA3B462A4621462846009600F079
:1026F00084FB43462A462146204600F06AFB3B46BF
:10270000224621462846009600F027FA3B460096CE
:102710002A462146204600F020FA2368DB074AD5E6
:1027200033463A462146204600F0BAF93146824601
:10273000204600F01CFD06F18043013B54F82300C5
:1027400040EACA7044F8230042462146284600F079
:1027500050FB3B460AAA29462846009600F04DFB4E
:102760003B460AAA29462846009600F046FB0AA9DD
:1027700008463B462A46009600F03FFB43460AAA1D
:102780002146204600F025FB02AA3B461046214682
:10279000009600F032FB32462946204600F0F4FC59
:1027A0004946284600F0F0FC02A9484600F0ECFC3F
:1027B00012B0BDE8F0873146204600F0D8FCC3E7F0
:1027C0000048704750D707002DE9F04FEDB01F4685
:1027D000DDF8D8810590B8F9026098F9004020230F
:1027E0001F3696FBF3F676B206F1FF3924AB0025CF
:1027F00043F829506CAB03EB89034CA88A469346F7
:10280000394698F9012043F8805C43F8605CFFF793
:10281000E1FE98F9012054A8B918FFF7DBFE214624
:102820004CA800F08BF90746002840F02E8154A8F0
:1028300000F084F90290002840F0298108F1240377
:1028400032464CA91846039300F063F9012840F082
:102850002081324654A9039800F05BF901280690C4
:1028600040F017811CAD0CAF3346039A54A928469B
:1028700000F08CF9029B47F829305A4651463846F9
:102880004346FFF7B1FE39463846039B00962A4679
:1028900000F0FFF90DF5B879039B00962A464CA984
:1028A00014A800F0F6F922464846059900F06CFCA1
:1028B000A30009EB030A0793059BA100591808F12F
:1028C000440B504600F060FC594634A800F05CFC14
:1028D000A3000BEB03013CA800F056FC08F1040335
:1028E000494634AA28460094049300F086FA5346D9
:1028F0004A463CA934A8CDF80080FFF7E7FD2346FF
:10290000049A2946284600F041F92A46514648468D
:102910004346FFF740FE029BCDE9083B059B31464D
:102920003846CDE90A3900F003FC3146814614A847
:1029300000F0FEFB8145B8BF81461FFA89F909F115
:10294000FF3B0FFA8BFB5946384600F059FC5946BD
:10295000071C14A818BF012700F052FC002814BF60
:10296000022300231F430DF1200A22465AF8277044
:1029700024A8394600F008FC0DF1B00BA300F918AB
:10298000584600F001FC2146284600F0B7F8A9F1AE
:102990000209069B2B600FFA89F90DF1900AB9F133
:1029A000000F23DA2346049A2946284600F0EEF861
:1029B00043462A4659465046FFF7EDFD32465146FA
:1029C000039800F0A6F8012804D03346039A504635
:1029D00000F0E6FB013C64B24CAA23064BD5029BF7
:1029E000B3FA83F040096DB0BDE8F08F43462A4644
:1029F000D8F8A47059465046B84749460CA800F08C
:102A0000FFFB4946071C14A818BF012700F0F8FB7C
:102A1000002814BF022300231F4308AB53F827707C
:102A200027B32246394634A800F0AEFB079B3CA8EA
:102A3000F91800F0A9FB43462A463CA934A8FFF741
:102A4000AAFD049B009434AA514644A800F0D5F98D
:102A50005B4652463CA934A8CDF80080FFF736FD0E
:102A6000434644AA2946284600F0B3F909F1FF3944
:102A70000FFA89F993E752F824105AF824304B40A2
:102A8000029919430291013CA7E72846ABE7384673
:102A9000A9E70298A7E7000000000000000000007E
:102AA000C3F10803DB0070B50133002403A500BFA8
:102AB0005B1920C940CAAD1920C0184720C940CAB7
:102AC000754120C020C940CA754120C020C940CAF4
:102AD000754120C020C940CA754120C020C940CAE4
:102AE000754120C020C940CA754120C020C940CAD4
:102AF000754120C06441204670BD00BF002310B561
:102B00001C465AB2914200DC10BD40F8234001330C
:102B1000F7E710B5013A52B2130601D5002010BDF7
:102B200050F8224051F822309C4205D802F1FF3281
:102B3000F2D24FF0FF30F2E70120F0E710B50023AA
:102B40001A465CB2A14203DCB2FA82F0400910BD21
:102B500050F8234001332243F3E770B59DF910404C
:102B60001E4623460546FFF79BFF30B922462946FD
:102B70003046FFF7CEFF012807D0234632462946CC
:102B80002846BDE8704000F00BBB70BDF0B50F46A5
:102B9000A1B006461946384615461C46FFF7CEFF3B
:102BA00020B13046FFF7AAFF21B0F0BD22463946DA
:102BB000684600F0E9FA294608A800F0E5FA10A8EE
:102BC0002146FFF79BFF012318A81093FFF796FFFC
:102BD000224608A96846FFF79CFF28B9224610A99B
:102BE000304600F0D1FADFE7009BDA0709D421462E
:102BF000684600F0BCFA2246294610A800F0E0FB27
:102C0000E6E7089BDB0707D4214608A800F0AFFAE7
:102C10002246294618A8F1E7002823461CDD08AA09
:102C20006946684600F0BCFA2146684600F09FFA03
:102C3000224618A910A8FFF76CFF002805DA10A992
:102C400023462A460846FFF72BFF10A9234618AA59
:102C5000084600F0A5FACEE708A96A46084600F043
:102C60009FFA214608A800F082FA224610A918A867
:102C7000FFF74FFF002805DA18A923462A46084621
:102C8000FFF70EFF18A9234610AA084600F088FA9D
:102C9000BEE72DE9F04FB5B004AD9DF9F8401F46F1
:102CA00081462346284600F0BAF824AB2146384630
:102CB000CDE9023500F03CFAC0EB841005B26B425E
:102CC00003F01F034FF0200695FBF6F676B205F0F1
:102CD0001F0814A858BFC3F100083146FFF70EFFC4
:102CE000B8F1000F30B22DDD14AB002203EB8000F1
:102CF000C8F1200C1346A34219D327B27B000193DD
:102D000014AB03EB870704F1FF3834AB012603EB68
:102D10008808002D53DA34AB03EB8606224656F8BA
:102D2000C81C484600F030FA35B0BDE8F08F57F8BF
:102D3000236006FA08F10A4340F8232026FA0CF231
:102D40000133D8E714AB2246394603EB800000F08C
:102D50001BFAD2E70FFA82FE5AF8C83C53F82EB09D
:102D600034AB03EB820252F8803CABEB03031B1A3B
:102D70009B4502D034BF012000205CF8C82C42F8EB
:102D80002E300131019B4AB29A42E3DB331A5E4294
:102D9000214614A85E4100F0EAF934AB03EB84034A
:102DA000214653F8802C58F8803C384643EAC273D9
:102DB000013D48F8803C2DB200F0D9F9A9E734ABC9
:102DC0000021C6F1010C084603EB860A03EB8C0CCC
:102DD000D8E730B51C4691B0054693F900306846F7
:102DE00000F01DF8D4F8AC3069462846984711B079
:102DF00030BD13460A46FFF7ECBF70B59DF9104091
:102E00001E462346054600F0CBF938B1234632462C
:102E100029462846BDE87040FFF742BE70BD2DE947
:102E2000F04F08B4F8CA04B451F8042BA3FB02898C
:102E300040F8048B4FF0000AE4FB629A4FF0000B5D
:102E4000E5FB62AB4FF0000CE6FB62BC4FF0000EFE
:102E5000E7FB62CE51F8042B4FF00008E3FB6289D8
:102E600040F8048BE4FB629AE5FB62ABE6FB62BCD4
:102E7000E7FB62CE51F8042B4FF00008E3FB6289B8
:102E800040F8048BE4FB629AE5FB62ABE6FB62BCB4
:102E9000E7FB62CE51F8042B4FF00008E3FB628998
:102EA00040F8048BE4FB629AE5FB62ABE6FB62BC94
:102EB000E7FB62CE51F8042B4FF00008E3FB628978
:102EC00040F8048BE4FB629AE5FB62ABE6FB62BC74
:102ED000E7FB62CE40F8049B40F804AB40F804BB2B
:102EE00040F804CB40F804EB0CBC052B00F01E812D
:102EF0000C68A0F11400A1F11401A2F1140252F81F
:102F000004EB4FF0000550F8046BE4FB6E5652F8EA
:102F100004EB50F8047BE4FB6E6752F804EB50F8C6
:102F2000048BE4FB6E7852F804EB50F8049BE4FB4E
:102F30006E8952F804EB50F804ABE4FB6E9AA0F1F2
:102F4000140052F8044B51F804EB4FF0000CE4FB72
:102F50006EC540F804CB51F804EBE4FB6E5640F824
:102F6000045B51F804EBE4FB6E6740F8046B51F826
:102F700004EBE4FB6E7840F8047B51F804EBE4FBCF
:102F80006E8940F8048B51F804EBE4FB6E9AA0E8DC
:102F90000006062B00F0CA800C68A0F11800A1F111
:102FA0001801A2F1180252F804EB4FF0000550F896
:102FB000046BE4FB6E5652F804EB50F8047BE4FB20
:102FC0006E6752F804EB50F8048BE4FB6E7852F80D
:102FD00004EB50F8049BE4FB6E8952F804EB50F8C4
:102FE00004ABE4FB6E9A52F804EB50F804BBE4FB2C
:102FF0006EABA0F1180052F8044B51F804EB4FF0FF
:10300000000CE4FB6EC540F804CB51F804EBE4FB84
:103010006E5640F8045B51F804EBE4FB6E6740F831
:10302000046B51F804EBE4FB6E7840F8047B51F834
:1030300004EBE4FB6E8940F8048B51F804EBE4FBED
:103040006E9A40F8049B51F804EBE4FB6EABA0E8E9
:10305000000C072B6AD008B40C68A0F11C00A1F189
:103060001C01A2F11C0252F804EB4FF0000550F8CD
:10307000046BE4FB6E5652F804EB50F8047BE4FB5F
:103080006E6752F804EB50F8048BE4FB6E7852F84C
:1030900004EB50F8049BE4FB6E8952F804EB50F803
:1030A00004ABE4FB6E9A52F804EB50F804BBE4FB6B
:1030B0006EAB52F804EB50F804CBE4FB6EBCA0F10D
:1030C0001C0052F8044B51F804EB4FF00003E4FBF2
:1030D0006E3540F8043B51F804EBE4FB6E5640F8C3
:1030E000045B51F804EBE4FB6E6740F8046B51F8A5
:1030F00004EBE4FB6E7840F8047B51F804EBE4FB4E
:103100006E8940F8048B51F804EBE4FB6E9A40F8AA
:10311000049B51F804EBE4FB6EAB40F804AB51F8B0
:1031200004EBE4FB6EBCA0E8001808BCBDE8F08F1F
:10313000013949B20A06CBB205D4013900EB81024C
:103140005268002AF6D001335BB273B103F18042BA
:10315000013A50F82220002022B9013B00EB431332
:1031600018B2704752080130F6E71846704700EB76
:1031700081010023884200D3704751F8042D43EAAF
:1031800052030B60D307F5E710B500235CB2A242EF
:1031900000DC10BD51F8234040F823400133F5E72F
:1031A000C3F10803DB0070B50133002403A500BFA1
:1031B0005B1920C940CAAD1B20C0184720C940CAAE
:1031C000B54120C020C940CAB54120C020C940CA6D
:1031D000B54120C020C940CAB54120C020C940CA5D
:1031E000B54120C020C940CAB54120C020C940CA4D
:1031F000B54120C06441B4FA84F0400970BD00BFFD
:103200004A11012350F8220001F01F0103FA01F1D5
:1032100008407047F0B5082289B00C460646FFF713
:10322000B3FFCB6A03930B6B04934B6B05938B6BD0
:103230000693CB6B0793002708236A4669466846C6
:10324000CDE901770097FFF72BFC082305466A4676
:1032500031463046FFF724FC236B0393636B0493E2
:10326000A36B0593E36B0544CDE906376A46082353
:1032700069466846FFF714FC082305446A46314650
:103280003046FFF70DFC236A0093636A0193A36A3B
:103290000293A36B0693E36B0793054408236A46E6
:1032A00031463046CDE904770397FFF7F9FB636AAF
:1032B0000093A36AA26B0193E36A02930492636B87
:1032C000E26B0393CDE90523236A079305440823A2
:1032D0006A4631463046FFF7E3FBE36A0093236B0F
:1032E0000193636B0293236A0693A36A07930544D1
:1032F00008236A4631463046CDE904770397FFF745
:103300004FFF236B0093636B0193A36B0293E36BFB
:103310000393636A0693E36A07932D1A08236A46A8
:1033200031463046CDE90477FFF73AFF636B0093EF
:10333000A36B0193E36B0293236A0393636A049381
:10334000A36ACDE90537236B07932D1A08236A4634
:1033500031463046FFF724FFA36B0093E36BCDE9C2
:103360000137636A0393A36A0493E36ACDE90537DF
:10337000636B07932D1A08236A4631463046FFF7E0
:103380000FFF2D1A0D4C0FD435B9082231462046B7
:10339000FFF7BFFB01280FD00823224631463046F5
:1033A000FFF7FEFE2D1AEFE708232246314630468E
:1033B000FFF776FB2D18F7D409B0F0BD54D70700FE
:1033C00070B5036813F001050646144605D0134690
:1033D0000A460146FFF764FB054621463046FFF7E3
:1033E000C6FE45B104F18042013A56F8223043F05E
:1033F000004346F8223070BD2DE9F0438BB00446FF
:10340000154689460AAE1C22002103A8FFF725F8BD
:10341000032346F8203D95F900802A464946204678
:103420002F1DFFF7E6FC3B46324621462046CDF8ED
:103430000080FFF7E2FC2B464A4621462046FFF774
:10344000C8FCCDF800803B4605F1840221462046A9
:10345000FFF783FB0BB0BDE8F08300002DE9F041DE
:103460001E4E4FF48271D6F8040130B11C48C26878
:10347000521CC260304605F0C9FD00254FF4A0770C
:1034800007EB85018AB23046B25812B389B205F013
:10349000BDFD1348103000EB0514204608F0F2FB88
:1034A000104811492246401AC008042101EB00408F
:1034B0000EA105F06DFB616819B1204608F038FBDC
:1034C00007E0A16811B1204608F032FB206800B186
:1034D00080476D1C022DD3D3BDE8F081004002402F
:1034E000F42A002088D8070038D8070074696D6571
:1034F000725F66697265202830782578290000009F
:1035000000F0DAB870B50E46144900EB400001EB4C
:10351000C0051446E86A183520B101280FD00228EA
:1035200005D113E0284600F0FDF8A04201D20024A6
:1035300011E022463146284600F02CF90BE02846DF
:1035400000F0F0F8A042F4D20446F2E731462846F3
:1035500000F0F3F80446204670BD0000F862002039
:1035600005F02EBF10B54FF080520023D2E94C1069
:103570000D2906D18C07C4F80C31C4F810313F4C2A
:1035800023600D2955D13E4B1B683E4C23603C4BBC
:103590001B1D1B68241D2360394B08331B68241D29
:1035A0002360374B0C331B68241D2360344B1033CE
:1035B0001B68241D2360324B14331B68241D2360B9
:1035C0002F4B18331B682F4C203423602C4B1C339B
:1035D0001B68241D23602A4B20331B68241D236095
:1035E000274B24331B68241D2360254B28331B687D
:1035F000241D2360224B2C331B68241D2360204B89
:1036000030331B681F4C403423601D4B34331B6820
:10361000241D23601A4B38331B68241D2360184B6C
:103620003C331B68241D2360154B40331B68241D4D
:1036300023600D2906D114480168C90702D06FF034
:10364000010101601148016841F470010160BFF39C
:103650004F8FBFF36F8FD2E94C010D2809D141B1D3
:10366000012906D04FF01020D0F80802034920317C
:10367000086008490648086010BD00003805004091
:103680000404001020C500400004004088ED00E064
:103690000090D003F02B0020064808B500210160FF
:1036A0000068009005F028FB05F0FEF80028FBD12B
:1036B00008BD00000001014010B5124C022020613D
:1036C000606111A0A06104F17800E0614FF48050C6
:1036D00020620020A06260620BA1A164E0620D493B
:1036E000E1641021A065C4E91410E0650AA1E01DA1
:1036F000FEF7D0FE09A12046FEF7CCFE2020A071E7
:1037000010BD0000F86200205465726D696E616C36
:103710000000000070730020525454005345474786
:10372000455200000269C1688A4203D88068401A85
:10373000104400E0501A401E70472DE9F047C4685D
:103740001746894606464FF000083069A04201D965
:10375000051B02E0B168201A0D1AB0686D1E001B2F
:10376000A84200D80546BD4200D33D4670682A46AF
:1037700020444946FEF756FEB0687F1B2C44A844FF
:10378000A944A04200D10024F460002FDDD14046BE
:10379000BDE8F0872DE9F04104468846D4E90207E8
:1037A000C51BE168606816460844B54206D9414623
:1037B000FEF738FEB819E060BDE8F0812A464146C0
:1037C000FEF730FE761B08EB050132466068FEF717
:1037D00029FEE660F0E702E008C8121F08C1002ACF
:1037E000FAD170477047002001E001C1121F002A82
:1037F000FBD170470121202803DA814005480140B0
:1038000003E0402802DA2038814009B101207047E6
:1038100000207047FC06FFBD800701D000207047E4
:103820000120704740680068401E084201D1012015
:10383000704700207047C3688B4206D81144006966
:10384000491E814201D801207047002070470000C6
:1038500030B585B00D46164C1621ADF800101ECCC3
:103860000DF1040C8CE81E00124C02210122217083
:103870006270A0700320E070217159206071FE20F9
:10388000A071694604F109007DDF00280ED1BDF862
:1038900000002A46411CE17109212172BDF808107F
:1038A0000844ADF8080001A9034872DF05B030BD37
:1038B000C0C20700283000202C2B002010B586B095
:1038C000062418220D496846FEF7ACFD0C480D4948
:1038D000401AC008042101EB00400BA105F054F987
:1038E00069462046FFF7B4FF002805D10A4C20782E
:1038F00074DF0121207873DF06B010BDD0C207004D
:1039000040D8070038D8070041647665727469733F
:10391000696E672E2E2E00002C2B00202DE9F05F03
:10392000DFF89CB05C46DBF84890DBF8246002F0DE
:1039300069FF216B4718751A22482349401AC108AC
:10394000042000EB0140804620A105F01DF9216B09
:103950004944B94200D1002508232A46384601F0DF
:103960002FFD0700184817494FF0010AA1EB00008E
:103970004FEAD0010AEB014404D020461AA105F019
:1039800003F919E002F03EFF0022314601F062F92E
:10399000DBF828200546D946AA4208D1404619A19D
:1039A00005F0F2F8C9E9075AC9F8186004E02046A2
:1039B0002B461A4905F0F3F83846BDE8F09F0000A1
:1039C000C047002088D8070038D80700456E7465C6
:1039D00072206E72665F6466755F6170705F636FA0
:1039E0006E74696E756500004661696C656420746B
:1039F0006F20636F7079206669726D776172652ED2
:103A00000000000053657474696E67206170702057
:103A100061732076616C696400000000F0C80700E3
:103A200008B51346024600930648074BC01AC00863
:103A3000012303EB00400B4604A105F0B8F806F0A3
:103A40009DFA000088D8070038D8070052656365E2
:103A5000697665642061206661756C7421206964F3
:103A60003A203078253038782C2070633A2030782E
:103A7000253038782C20696E666F3A2030782530F2
:103A800038780000024606480649401AC00801215D
:103A900001EB004004A105F07BF806F06FFA00008E
:103AA00088D8070038D80700526563656976656471
:103AB00020616E206572726F723A2030782530383E
:103AC000782100002DE9F04107461E4E1E481F498F
:103AD000326A401AC508012A04D0032000EB0540D1
:103AE0001BA12BE04FF44050184B174C4168E31AD0
:103AF000234A0220DB0800EB0344914206D1C102B5
:103B00003B462048726B00F04FFF90B102F07AFE06
:103B100001461C483B464130B26900F045FF58B1B0
:103B2000042000EB054018A105F02EF80120BDE8A7
:103B3000F081204618A101E0204626A105F024F8D6
:103B40000020F4E7C047002088D8070038D80700D5
:103B5000426F6F742076616C69646174696F6E2066
:103B60006661696C65642E204E6F2076616C6964B5
:103B70002061707020746F20626F6F742E000000DF
:103B8000DBE5B151204A0020417070206973207636
:103B9000616C696400000000426F6F742076616C94
:103BA00069646174696F6E206661696C65642E205A
:103BB000536F66744465766963652069732070721B
:103BC0006573656E742062757420696E76616C69C8
:103BD000642E0000426F6F742076616C69646174BA
:103BE000696F6E206661696C65642E20417070207B
:103BF000697320696E76616C69642E002DE9F84F57
:103C0000254C8146924660880E46814241D8002765
:103C10004FF6FF788DF80070684600F075F822784E
:103C20006078A188884201DA401C00E00020C0B220
:103C3000904204D19DF8000000F0B2F827E06578CA
:103C40006078884201DA401C00E0002060709DF836
:103C5000000000F0A5F8454519D0A068B9F1000FA3
:103C600040F835A00DD066B16188E068324605FBAA
:103C700001004946FEF7D6FBA06800EBC500868030
:103C800002E000EBC50087800020BDE8F88F04202B
:103C9000FBE70920F9E70000702B002010B50E4C5F
:103CA00003E0401C00E00020207020786178814211
:103CB00010D022786188E068A36802FB010003EB62
:103CC000C20153F83220898890472078A188884221
:103CD000E9DAE6E710BD0000702B002030B5CB001C
:103CE00008339DB293074FF0000401D0072030BD88
:103CF000044B9A602A44DA605C701C70588099808A
:103D0000002030BD702B002070B5044606F0FEFF89
:103D1000012803D010A1432000F086F8EFF31081B2
:103D200072B61D4A9368012083B990604FF0E0207D
:103D3000D0F88051194B1D401560C0F88031D0F883
:103D4000843153604217C0F884210020207000297C
:103D500000D162B670BD00002E2E5C2E2E5C2E2E81
:103D60005C2E2E5C2E2E5C636F6D706F6E656E74B4
:103D7000735C6C69627261726965735C7574696C9D
:103D80005C6170705F7574696C5F706C6174666F94
:103D9000726D2E6300000000344F0020FC06FFBD52
:103DA00010B5044606F0B2FF012803D00DA1512042
:103DB00000F03AF81B498868002811D0002C0FD178
:103DC000EFF3108072B60B684FF0E022C2F80031BA
:103DD0004B68C2F8043100228A60002800D162B624
:103DE00010BD00002E2E5C2E2E5C2E2E5C2E2E5C26
:103DF0002E2E5C636F6D706F6E656E74735C6C6994
:103E0000627261726965735C7574696C5C61707013
:103E10005F7574696C5F706C6174666F726D2E6330
:103E200000000000344F00201CB56A46CDE90001B7
:103E3000002144F20200FFF7F3FD1CBDF8B5214854
:103E40000146456AC06A8C6CAC2801D024B106E0FA
:103E5000486B04442D1A02E002F0E8FC04461A48BC
:103E60001A492346401AC708042000EB07400646BB
:103E7000174A18A1009504F09AFE2A4621461448D4
:103E8000FEF7FBFAD0B130462B4622461FA104F0C4
:103E900086FE00BF04F008FD0028FBD102F086FA80
:103EA0002946204603F0AAF8040005D0012000EBC3
:103EB000074022A104F068FE2046F8BD00243046E9
:103EC00025A1F7E7C047002088D8070038D80700A9
:103ED00000200700566572696679696E6720424C5A
:103EE0003A20416464723A203078253038782C20AA
:103EF0005372633A203078253038782C204C656E28
:103F00003A2030782530387800000000436F70790F
:103F1000696E6720626F6F746C6F616465723A20BE
:103F20005372633A203078253038782C204C656EF7
:103F30003A203078253038780000000052657175DD
:103F400065737420746F20636F707920424C206613
:103F500061696C65640000004E6F20626F6F746C65
:103F60006F6164657220636F7079206E656564654A
:103F7000642C20626F6F746C6F6164657220757061
:103F80006461746520636F6D706C6574652E0000EC
:103F900030B595B0040004D12E4940F24F40FFF7F0
:103FA00043FF2D494FF6FF702246488001208DF8CF
:103FB00012004FF65960ADF8100004A90120A8DFE7
:103FC000002844D1254B0FCB8DE80F00A11C68467B
:103FD00062DF00283BD121491C2260390BA8FEF783
:103FE00021FA1F4D142205F1C401A8681290A0788F
:103FF0008DF84A002868139006A8FEF713FA12A855
:10400000069013A807902088231D06AA0BA9AADFF3
:1040100000281CD11C2205F1D8010BA8FEF702FADA
:10402000E8681290A0788DF84A006868139014220E
:1040300005F1F40106A8FEF7F5F912A8069013A8F9
:104040000790208804F10C0306AA0BA9AADF15B07B
:1040500030BD0000DCC907002C2B002098C30700EE
:1040600090C20700F0B585B00D46040004D1374971
:1040700040F28710FFF7D8FE25B934494FF4C470D9
:10408000FFF7D2FE14216846FEF7E5F920780323F6
:1040900008280BD12E48C188491E89B2C180828868
:1040A000002A4BD0002949D1C28023702178607842
:1040B00060228DF800208DF801108DF802006378E1
:1040C0000325012B16D0234823492278401AC00823
:1040D000022101EB004021A104F061FD60780B2872
:1040E00028D101F0ADF88DF80300002001F0B0F800
:1040F00004251FE0207809281CD2DFE800F01B1BF4
:104100001B211B1B051B2100D4E902706D46E91C15
:10411000666807F0DDFD044629193046C91C07F022
:10412000D7FD044429193846C91C07F0D1FD2044A5
:10413000C01CC5B22946684606F0B0FE05B0F0BD09
:10414000D4E90112684606F098FEF1E7DCC90700E1
:104150002C2B002040D8070038D8070044465520B3
:1041600072657175657374202564206661696C657C
:10417000642077697468206572726F723A203078B3
:10418000257800002DE9F0411D4C0026217AC90751
:1041900033D01C49884230D01B481C49401AC10802
:1041A000042000EB0140054619A104F0EDFC6088F5
:1041B000A0F57F41FF3916D028461DA104F0E4FC8C
:1041C000A068132140F00400A060608876DF00281A
:1041D00014D11B4CC8264FF47A47611C38468847D7
:1041E000761EFAD101E0207874DF05F085F806002C
:1041F00003D1284613A104F0C7FC3046BDE8F08186
:104200002C2B002020D8070040D8070038D8070002
:104210005368757474696E6720646F776E20424CC2
:1042200045207472616E73706F72742E000000000E
:10423000446973636F6E6E656374696E672E000008
:10424000A0C20700424C45207472616E73706F7299
:1042500074207368757420646F776E2E0000000000
:1042600070B5204C06460020217AC90738D11E4877
:104270001E49401AC108042000EB014005461CA15C
:1042800004F082FC2248E66001F012FD00F01CFB05
:10429000002825D103F088F838B11E4803F078F8DB
:1042A000A06840F00200A06003E028461AA104F0D4
:1042B0006BFC01F019F8002812D116481C30FFF7EA
:1042C00067FE00280CD1FFF7F9FA002808D1A06892
:1042D00018A140F00100A060284604F055FC002021
:1042E00070BD00002C2B002040D8070038D80700F4
:1042F000496E697469616C697A696E6720424C45E0
:1043000020444655207472616E73706F72740000A1
:10431000A8D80700483000204E6F2061647665728F
:10432000746973696E67206E616D6520666F756E66
:1043300064000000424C4520444655207472616E72
:1043400073706F727420696E697469616C697A65E3
:10435000642E00002DE9FE439F49A04B0122591A0B
:10436000C9080746051D02EB0148008804229C4E3F
:104370004FF0000902EB014421286ED037DC1328EE
:104380006CD01EDC01286AD0102854D0112868D0C7
:10439000122879D1204693A104F0F6FBEA88204642
:1043A0009AA104F0F5FBAA8820469EA104F0F0FB38
:1043B0002A892046A1A104F0EBFB6A892046A4A12A
:1043C000ECE0142875D01A2874D01F285CD1204640
:1043D000A5A104F0D9FB291D708875DF040053D016
:1043E00040462246ACA104F0D3FB20461FE05128F2
:1043F0007AD00EDC222878D0232868D024287BD0DD
:10440000502877D103B03946BDE8F043B04805F0F5
:1044100045BE5228D8D0552837D056286AD1B87909
:10442000002867D11321708876DF002862D0BDE8AC
:10443000FE43FFF727BB2046A6A104F0A5FB288872
:104440007080F16809B101208847A549708875DF3F
:1044500002004FD04046A3A1A0E07FE055E087E0F6
:10446000FFE74FF6FF707080307A400704D4FFF703
:1044700025FA08B1FFF706FBF16800293AD003B02E
:104480000220BDE8F043084734E0FA88F72A14D246
:104490009007B0F1404F0ED0D01F81B2481EC31715
:1044A00000EB937323F00303C01A081A801D85B232
:1044B00004E078E081E0154600E0F72520462B4631
:1044C000944904F06CFB29467088B5DFADE72046BF
:1044D00091A104F059FBCDF80090CDF80490B88874
:1044E0000022694690DF2DE046E02EE004E000BFA8
:1044F000FFF7C8FABDE8FE836B89EA8803B020465F
:10450000BDE8F04391A104F04ABB20469FA104F00E
:104510003BFB734801AA163842F60521806A0190D8
:10452000CDF808D07088ADDF08B1FFF7ABFA2046B0
:10453000BDF800209FA104F02BFB00231A46852123
:1045400070887FDF0028D3D1D4E7287900906B7979
:10455000AA792046A0A104F02AFBCBE72046ADA112
:1045600004F012FBCDF80090288869468FDFE9E758
:104570000021708866DF58E7B8790028BAD039463C
:10458000534805F047FD0028B4D007F10801504812
:1045900005F060F90200ADD04046A9A103B0BDE826
:1045A000F04304F0F5BA2046B2A104F0EDFA002180
:1045B0000A4628880B4686DF37E7002328881A46F4
:1045C0001946B1DF08B1FFF75DFA03B02046BDE838
:1045D000F043B2A104F0D8BA38D8070040D8070099
:1045E0002C2B0020526563656976656420424C453A
:1045F0005F4741505F4556545F434F4E4E5F5041B9
:1046000052414D5F55504441544500006D61785F03
:10461000636F6E6E5F696E74657276616C3A2025A9
:10462000640000006D696E5F636F6E6E5F696E742B
:10463000657276616C3A202564000000736C6176C7
:10464000655F6C6174656E63793A202564000000D3
:10465000636F6E6E5F7375705F74696D656F75748F
:104660003A20256400000000526563656976656440
:1046700020424C455F4741505F4556545F434F4E83
:104680004E5F504152414D5F5550444154455F5239
:1046900045515545535400004661696C757265205B
:1046A000746F2075706461746520636F6E6E6563EE
:1046B00074696F6E20706172616D657465722072CD
:1046C0006571756573743A203078257800000000B4
:1046D00064300020436F6E6E656374656400000093
:1046E000A6C207004661696C75726520746F2075FB
:1046F000706461746520636F6E6E656374696F6E5C
:1047000020706172616D65746572733A203078252E
:104710007800000094C90700526563656976656496
:1047200020424C455F4741505F4556545F444154D9
:10473000415F4C454E4754485F5550444154455F96
:10474000524551554553542E000000005265636593
:104750006976656420424C455F4741505F45565439
:104760005F444154415F4C454E4754485F55504467
:10477000415445202825752C206D61785F72785F43
:1047800074696D65202575292E00000052656365EA
:104790006976656420424C455F4741505F455654F9
:1047A0005F5345435F504152414D535F5245515510
:1047B000455354004343434420666F72207365722F
:1047C00076696365206368616E676564206973203C
:1047D0003078253034780000526563656976656409
:1047E00020424C455F4741505F4556545F50485901
:1047F0005F555044415445202852583A25642C2096
:1048000054583A25642C207374617475733A256486
:1048100029000000526563656976656420424C4555
:104820005F4741505F4556545F5048595F5550446B
:104830004154455F524551554553542E00000000E8
:10484000436F756C64206E6F742068616E646C6574
:10485000206F6E5F6374726C5F70745F77726974DF
:10486000652E206572725F636F64653A203078252B
:1048700030347800526563656976656420424C4542
:104880005F4741505F4556545F5345435F494E462D
:104890004F5F5245515545535400000046696E69BB
:1048A000736865642068616E646C696E6720636F0D
:1048B0006E6E20736563207570646174650000001E
:1048C000007800F00100704738B50020009002F039
:1048D000A1FB00282DD117481749184A401AC108D2
:1048E000042000EB0140044615A104F051F91348DF
:1048F00013DF00281DD1204619A104F045F904F06A
:1049000025FD002815D1684604F086FB002810D14B
:10491000204619A104F038F96946012004F086FB0D
:10492000002806D120461AA104F02EF9684604F0AA
:1049300015FC38BD40D8070038D807000020070014
:1049400053657474696E6720757020766563746F43
:1049500072207461626C653A2030782530387800B6
:10496000456E61626C696E6720536F66744465764C
:104970006963652E00000000436F6E66696775729B
:10498000696E6720424C4520737461636B2E000092
:10499000456E61626C696E672074686520424C45A3
:1049A00020737461636B2E0013B90378012B01D05F
:1049B00002F06CBF012070470022C32100F518707F
:1049C00000F048B92DE9F043A1B00446DDE928968E
:1049D00020200F46209098461546782102A8FDF722
:1049E0003AFD41212046FDF736FDB7F8940005EB6E
:1049F000051107EB8101A84201D991F89660267054
:104A0000320033D0012A0DD01B481C4D0123401B1E
:104A1000C00803EB0045022A0CD0032A20D0284608
:104A200017A117E000224946404600F013F9C4F8E8
:104A300001001BE020A9601CCDE900014B46424665
:104A4000184902A801F0B0FD80B104F0B1FD0246A2
:104A5000284615A104F09CF8002021B0BDE8F083A1
:104A6000B1F89820601C9A31FDF7DCFC4A464146BB
:104A7000204602F00BFFF0E768D8070038D807009F
:104A8000496E76616C696420626F6F742076616C28
:104A900069646174696F6E20747970653A20256469
:104AA00000000000B8C007006E72665F6372797024
:104AB000746F5F686173685F63616C63756C617468
:104AC000652829206661696C6564207769746820AF
:104AD0006572726F722025730000000010B50446E5
:104AE0000A480B49401AC008042101EB004009A103
:104AF00004F04AF84FF0000034B10C490870BDE8EA
:104B000010400B4802F07CBC00F0E2FA88D80700A5
:104B100038D80700526573657474696E6720626FD8
:104B20006F746C6F616465722E000000E82A0020CB
:104B3000D15007002DE9F84F0546861C00208DF85E
:104B4000000091460F464FF0010A6846FFF7DCF877
:104B50001C4C60683860D4E901011B4F401A396869
:104B6000081A41F21C0104EB01080EE00121404645
:104B700000F0C9FF00F01EFE0146404600F0C3FFF2
:104B8000D4E90101401A3968081A401C8642EDD860
:104B9000B9F1000F03D0052065F3891002E006206B
:104BA00065F39F5061683A68114004EB8101C86069
:104BB0006068304460609DF80000FFF7F1F85046EF
:104BC000BDE8F88FD8520020982B002010B543681C
:104BD0009C18446021B905E013F8010B01F8010BA2
:104BE000521EF9D2012010BD70B50D4604460A29A7
:104BF00002D10D21FFF7F8FFA0682268411CA160D7
:104C00001554D4E90101814204D32046BDE8704027
:104C100003F088BA70BD0000044881684068814292
:104C200001D101207047002070470000D8520020B9
:104C300010B5040003D10549F020FFF7F5F804484A
:104C4000C16B6160006CA06010BD0000DCCA070091
:104C5000C0470020F0B54FF0FF3622B11268D243B2
:104C600000230A4D0DE03246FAE7C45C6240082496
:104C7000D70700D037462F4087EA5202641EF7D18B
:104C80005B1C8B42F1D3D043F0BD00002083B8ED14
:104C900010B504460068401C07D0204606F05EFBB5
:104CA0002168814201D1012010BD002010BD00000B
:104CB00010B5104C90B06078002818D101F0D8FCE5
:104CC00018B10D49DB20FFF7AFF820220B496846E9
:104CD00001F0EEFC40236A4609490A4801F024FC31
:104CE00018B10549E520FFF79FF80120607010B06A
:104CF00010BD0000602B0020BCCE070058C007008C
:104D00006C4E0020D0C00700F0B5146906468DB087
:104D100020681546271DE0B1022920D00A20009006
:104D20006B4609AA304606F077F800280FD009A98B
:104D300001A8009A05F09CFD01AE96E80F0005AEB3
:104D400086E80F00236869683A4605A898470DB0C1
:104D5000F0BD0DB03046BDE8F04005F0FDBD694640
:104D6000304605F08FFD0028F1D0236869683A4687
:104D7000684698470028EAD002980028F5D10198A3
:104D800070600120E3E753689B7813F0C00303D001
:104D9000402B03D00020704700F002B8FFF7B4BFEB
:104DA0002DE9FF410B465168064614468878334D7D
:104DB00000F00F0210F0300055F8225006D01028F5
:104DC00006D0202808D0302856D13EE022694DE098
:104DD00061690120087047E0022B28D1042A26D8F7
:104DE0004FF0010869463046676905F04BFD002821
:104DF0001AD009E00B89226903FB00226846A84704
:104E000070B13888401C3880029820B161683888B9
:104E10004A899042EED301987060029860BB02E02C
:104E20004FF00008F7E7404604B0BDE8F081D4E950
:104E300004300F890288498907FB02338A421BD25A
:104E4000521C02801A46616810E008886169072ACE
:104E5000088009D1606801892069FDF7FCFA606863
:104E60002169C06805F029FD2269616804B03046F7
:104E7000AC46BDE8F04160470020D5E758C70700C1
:104E80001A4910B50A680120D20301D5000408E0D0
:104E900017490A6802F0F902A92A04D1086800F04B
:104EA000560008600020FEF70DFE1249124A891ACA
:104EB000C908042202EB014260B10D48001F0068DE
:104EC00000F0F900B12808D00C48806D012807D007
:104ED000002010BD10460AA104E0104611A101E017
:104EE000104619A103F050FE012010BD000400403F
:104EF0002005004088D8070038D80700C0470020A8
:104F0000444655206D6F6465206265636175736505
:104F100020617070206973206E6F742076616C69F7
:104F2000642E0000444655206D6F646520726571E3
:104F300075657374656420766961204750524547F2
:104F40005245542E00000000444655206D6F6465A4
:104F5000207265717565737465642076696120627D
:104F60006F6F746C6F616465722073657474696EC1
:104F700067732E00FEB519490446086808B1401E43
:104F800008601748174AD4E90153801AC008042260
:104F900002EB004022789DB10E6821690296CDE9AE
:104FA00000312B46012A16D00FA211A103F012FEE8
:104FB0006169002911D0E06803B0BDE8F0400847FE
:104FC00009680091012A04D007A218A103F0EFFD9F
:104FD000EEE720A2F9E71FA2E7E7FEBD442B002081
:104FE00048D8070038D80700657261736500000073
:104FF000466C617368202573206661696C65642066
:105000002830782578293A20616464723D25702C17
:10501000206C656E3D307825782062797465732C3C
:105020002070656E64696E6720256400466C61734C
:105030006820257320737563636573733A20616418
:1050400064723D25702C2070656E64696E67202542
:10505000640000007772697465000000704700000A
:1050600010B50446801E062810D2DFE800F00D03BC
:10507000030F09090A494FF4701000F087FF05E09B
:105080000120FFF72BFD01E002F046FA05484168D8
:10509000002903D02046BDE81040084710BD00009D
:1050A00035550700E82A002010B50446062801D02F
:1050B000072C02D1002002F02BFB044801680029D4
:1050C00003D02046BDE81040084710BD282B002023
:1050D00003F012FE03F0E8FB0028FBD1BFF34F8F73
:1050E00005480168054A01F4E06111430160BFF31E
:1050F0004F8F00BFFDE700000CED00E00400FA0553
:1051000010B50021024800F014FD80F3100010BD1E
:10511000F46200202DE9FC4180461F4615460E46EC
:1051200000240D4800F0ECFC38B11120BDE8FC81F2
:1051300006EB043003F00AFF641CAC42F8D10648C9
:1051400000F0D5FCCDE9005733460022022140464D
:1051500000F02AF80020E9E7802B00202DE9F84331
:10516000104D0F4680461E4691466946286800F05D
:1051700092FC040014D01C21FDF76DF90120207170
:10518000C4F81490380BC4F80080C4E90260694682
:10519000286800F0A1FC05F01FFE0020BDE8F883A0
:1051A0000420FBE724C407002DE9F04387B0044640
:1051B000DDE90E8980681D4616460F4600280BD093
:1051C00018216846FDF747F902A88DF8007080E8BD
:1051D0006003A1686846884707B0BDE8F08330B532
:1051E0000446006887B00D46806800281FD018214B
:1051F0006846FDF730F90195A0680590207910B157
:10520000012810D107E001208DF8000020690290EC
:10521000E068039005E002208DF80000E0680003DC
:10522000029060690490206881686846884707B0EA
:1052300030BD0B2803D30B38C0B200F009B870475B
:105240000249002208780A7070470000482B0020AD
:10525000014908700B207047482B002001490120AC
:1052600008707047E82A0020014901200870704743
:10527000242B002070B515460E46040004D10749C2
:105280004FF42C70FEF7D0FD2A46314604F172002F
:10529000BDE87040012302F04BBB0000BCCE07000C
:1052A00010B5040003D10E49DB20FEF7BDFD2078C8
:1052B00018B90B49DC20FEF7B7FD94F855000949F1
:1052C00038B1012805D06068C968884205D9012035
:1052D00010BD606889688842F9D24FF0000010BDA7
:1052E00004CF0700C04700203EB59DF8080020F01D
:1052F0000F00401C20F0F00010308DF808006846C8
:105300006DDF00282BD19DF80100401C8DF80100B5
:1053100068466CDF002822D111481349007A8207C1
:105320001048A0EB01004FEAD0004FF0040101EB60
:10533000004008D50D4C0EA1221DA36903F02FFCDF
:10534000211DA06904E013A103F01EFC19A1072090
:1053500082B202A87CDF002801D118487ADF3EBD66
:105360002C2B002040D8070038D8070048300020F8
:1053700053657474696E6720616476206E616D6533
:105380003A2025732C206C656E6774683A2025647A
:10539000000000005573696E672064656661756C76
:1053A00074206164766572746973696E67206E61DA
:1053B0006D6500004466755461726700A6C20700FF
:1053C0002DE9FC5F164607463A4A3B481D46101A2F
:1053D00004224FEAD00902EB09408B468246B942CB
:1053E00005D136A103F0D0FB0020BDE8FC9F04D21C
:1053F00036494FF04F00FEF717FD1DB933495020D5
:10540000FEF712FD2EB1380503D030495320FEF7C8
:105410000BFDABEB0700040B03D12C495720FEF723
:1054200003FD0020009006F6FF704FEA103800F0F0
:10543000D1FFA54239D22C4637E0A04503D83546E6
:10544000CDF8048001E0250301940022384601993B
:1054500001F062FC0028C8D150463B465A461CA1C8
:10546000009503F0A4FB681E00F003002A1A002335
:1054700059463846D21C01F005FD0028B5D10199E6
:105480001C48A8EB0108761B016B2F4429440163DB
:10549000AB44002002F028F9009030B1012101EB6B
:1054A000094015A103F070FB01E0002EC5D1009862
:1054B0009BE7000088D8070038D807004E6F2063AC
:1054C0006F7079206E65656465640000A0C8070090
:1054D000436F7079696E67203078257820746F206B
:1054E000307825782C2073697A653A2030782578D1
:1054F00000000000C04700204661696C65642074AC
:105500006F20777269746520696D61676520636FCC
:105510007079696E672070726F677265737320743B
:105520006F2073657474696E677320706167652E90
:10553000000000000748084910B5401AC0080321C0
:1055400001EB004005A103F01FFBBDE81040012066
:10555000FFF7C4BA88D8070038D80700496E6163DE
:105560007469766974792074696D656F75742E003D
:105570000149416000207047F8C3070010B50B498E
:1055800041600B4800F0BCFA68B903F031FF0849EC
:105590001C234FF4EE7208740448A1F5EE71001F4D
:1055A000006800F065FA002010BD000028C4070064
:1055B0002C5100202DE9FC5F0E008346DDE90C47ED
:1055C000C6F1000098469246814600D4084601255F
:1055D00003E000BF90FBFAF06D1C5045FADAA845D5
:1055E00000D9454624B1002E01DB780700D5641EA2
:1055F000B80702D5B8F1000F0AD0F80708D13CB1BE
:10560000A54205D220215846641EFFF7EDFAF6E7C1
:10561000002E02DA4E462D2102E0780703D52B2119
:105620005846FFF7E1FA07F0030002280BD1B8F162
:10563000000F08D13CB1A54205D230215846641E66
:10564000FFF7D2FAF6E7CDE9004743465246314626
:10565000584606F05FFBBDE8FC9F0246002012683A
:10566000530713D502F00300012802D002280CD101
:1056700005E0C2F383100B68801C184404E0022389
:10568000086803EB92521044086001207047000044
:1056900002480068002800D001207047802B0020BD
:1056A0000248007A002800D0012070472C510020C9
:1056B00038B54FF440521B49536800F500508B42F7
:1056C00004D044688C4201D1012400E000248B42C4
:1056D00026D143688B4223D11178142901D952690C
:1056E00000E000221049B2FBF1F30278142A01D93C
:1056F000406900E00020B0FBF1F0834203D00124B8
:105700000AA2009002E000240AA200900B480C4973
:10571000401AC008032101EB00400AA103F047FA38
:10572000204638BDDBE5B15140420F006D616A6F24
:10573000720000006D696E6F7200000068D807008B
:1057400038D80700536F66744465766963652075C1
:10575000706461746520697320612025732076650B
:105760007273696F6E207570646174652E20437565
:105770007272656E743A2025642E204E65773A2049
:1057800025642E0070B5054608680C464A68866890
:105790002846314604F0B2FF6068286104F10C002D
:1057A0006861B0780221B1EB901F01D1241D2C61FA
:1057B00070BD70472DE9FF410026274800F09DF994
:1057C0002548001F074600F098F9244C2449A0689A
:1057D00000900D6800E000986946284004EB8000C6
:1057E0000C30FFF73AFF0028F5D101AA009901EA31
:1057F000050304EB8303491CDB6842F82030401C9E
:1058000000910228F2D3019800F0030001281AD079
:1058100002280ED013A14FF4C270FEF705FB3846E4
:1058200000F068F908B10098A06004B03046BDE807
:10583000F0810198032101EB90500099BDF80A60B6
:1058400001EB900005E00198BDF80A60C0F38310F9
:1058500008440090E3E70000F0620020D8520020E6
:10586000982B00202E2E5C2E2E5C2E2E5C2E2E5C75
:105870002E2E5C636F6D706F6E656E74735C6C69F9
:10588000627261726965735C6C6F675C7372635C92
:105890006E72665F6C6F675F66726F6E74656E6462
:1058A0002E63000000F06AFD4FF48051002000F0EC
:1058B0008DFBC8B91548C0F5FC2100F087FB98B9ED
:1058C0000021134803F0ECF902F0D8FF1148124907
:1058D000401AC408032000EB044010A103F054F95F
:1058E000114800F079FC08B1FEF7CCF802F0DCFFBB
:1058F0000028FBD1012000EB04400CA103F044F987
:1059000002F0D2FF0028FBD1EEE7000000200700E4
:10591000B55F070088D8070038D80700496E73695B
:105920006465206D61696E005D50070041667465B5
:1059300072206D61696E2C2073686F756C64206EC7
:105940006576657220626520726561636865642EA4
:10595000000000002DE9F05F1E46DDF828B09146FA
:105960008A46040003D124A1B620FEF75DFAB4F8FC
:105970000680607908FB00F8A8F10408464503D3C7
:105980001DA1C420FEF750FAE788301DB0FBF7F1E7
:10599000B0FBF7F207FB1200D9F80050AA194245F4
:1059A00001D9A8EB0605C9F8005001E02468491E9A
:1059B0000029FBD13E1A8846AE4215D817E000BF39
:1059C0002044001D0AEB0803BBF1000F324602D051
:1059D0000146184600E01946FCF724FD0020246823
:1059E000AD1BB044AF4201D92E4600E03E46002D2B
:1059F000E6D1BDE8F09F00002E2E5C2E2E5C2E2EF0
:105A00005C2E2E5C2E2E5C636F6D706F6E656E74F7
:105A1000735C6C69627261726965735C6D656D6FF0
:105A2000626A5C6E72665F6D656D6F626A2E63009E
:105A300030B5024651B103F047F90021074C08E0A8
:105A400034F821301568AB4202D11160002030BD1E
:105A5000491C8142F4D3052030BD00000000000045
:105A600010B5FCF724FC08B1002010BD112010BDBA
:105A700010B531B1B2FBF3F403FB14241CB10920BF
:105A800010BD0E2010BD0160002141608160828147
:105A9000C381084610BD70B50C460546FCF7BCFB3B
:105AA000002802D021882868084470BD10B50A88F3
:105AB00049888A4203D1FCF7F1FB012010BD002088
:105AC00010BD70B50C460546FCF7CBFB002802D094
:105AD00061882868084470BD10B50A8849888A42E0
:105AE00003D1FCF7B5FB012010BD002010BD002143
:105AF00000F00FB8002100F012B8012100F01EB82C
:105B0000012100F011B808B56A46FCF71CFC0098AA
:105B100008BD08B56A46FCF7FCFB009808BD08B54F
:105B20006A46FCF7F6FB08BD08B56A46FCF7E4FBDD
:105B300008BD08B56A46FCF7D3FB08BD08B56A4640
:105B4000FCF7DAFB009808BD08B56A46FCF708FCCC
:105B5000009808BD38B5040004D115A14FF4927027
:105B6000FEF762F900258DF800506846FEF7CCF884
:105B7000206862680168914214D9491E01600D785D
:105B80001CB919A1E820FEF74FF9208AE16805FB4E
:105B900000152068217A0278891A0279C9B28A42EE
:105BA00000D201719DF80000FEF7FAF8284638BDD2
:105BB0002E2E5C2E2E5C2E2E5C2E2E5C2E2E5C63EA
:105BC0006F6D706F6E656E74735C6C69627261721A
:105BD0006965735C62616C6C6F635C6E72665F6258
:105BE000616C6C6F632E63002E2E5C2E2E5C2E2E4D
:105BF0005C2E2E5C2E2E5C636F6D706F6E656E7406
:105C0000735C6C69627261726965735C62616C6C11
:105C10006F635C6E72665F62616C6C6F632E6300B3
:105C200038B50C46050004D112A140F24710FEF72A
:105C3000FBF824B90FA14FF4A470FEF7F5F800208B
:105C40008DF800006846FEF75FF81DB91749F5208A
:105C5000FEF7EAF8E8682A68211A288AB1FBF0F111
:105C60001068431C136001709DF80000FEF798F85F
:105C700038BD00002E2E5C2E2E5C2E2E5C2E2E5C4F
:105C80002E2E5C636F6D706F6E656E74735C6C69E5
:105C9000627261726965735C62616C6C6F635C6E89
:105CA00072665F62616C6C6F632E6300E85B070075
:105CB00010B5040002D0206830B901E00E2010BDFC
:105CC00019A1FF20FEF7B0F8606820B916A14FF4C3
:105CD0008070FEF7A9F8A06820B913A140F2011066
:105CE000FEF7A2F8E06820B90FA14FF48170FEF72B
:105CF0009BF8208A20B90CA140F20310FEF794F81B
:105D0000207A61682268401AC0B2116004E02268FB
:105D100011684B1C13600870401EC0B2F7D2216896
:105D20000020087110BD00002E2E5C2E2E5C2E2E41
:105D30005C2E2E5C2E2E5C636F6D706F6E656E74C4
:105D4000735C6C69627261726965735C62616C6CD0
:105D50006F635C6E72665F62616C6C6F632E630072
:105D60002DE9F041184819494FF48052401AC708EC
:105D7000042000EB0745164615A1284602F008FF4F
:105D80004FF0E024D4F8802128461FA104F5C07408
:105D900002F0FEFE60172060C4F800016060C4F8E5
:105DA000040101F043F928B1012000EB074021A1D3
:105DB00002F0EAFE02F078FD0028FBD13046BDE893
:105DC000F04100F053B8000088D8070038D8070029
:105DD00052756E6E696E67206E72665F626F6F7469
:105DE0006C6F616465725F6170705F73746172740F
:105DF000207769746820616464726573733A203037
:105E0000782530387800000044697361626C696EEF
:105E10006720696E74657272757074732E204E56A9
:105E200049432D3E494345525B305D3A2030782549
:105E3000780000004661696C65642072756E6E6959
:105E40006E67206E72665F6466755F6D62725F6911
:105E500072715F666F72776172645F6164647265AC
:105E600073735F73657428290000000070B50646DF
:105E70002648C0F5FE2100F0A9F804002448254971
:105E8000A0EB01004FEAD0004FF0010101EB00450B
:105E900007D02846224620A102F07AFE2046FDF7D0
:105EA000F1FD00F0AFFC014629488069421EC2F3B3
:105EB0000B02801A0144002001F6FF7100F086F801
:105EC000040004D02846224622A102F061FE201ED2
:105ED00001D0FDF7D7FDEFF30580C105D6E90045F8
:105EE000C90D4FF0000080F3148880F3108880F310
:105EF000118880F3138803D023495820FDF794FFBD
:105F000084F30888AC46BDE8704060470020070075
:105F100088D8070038D80700436F756C64206E6F0F
:105F2000742070726F7465637420626F6F746C6F2D
:105F30006164657220616E642073657474696E6754
:105F4000732070616765732C20307825782E0000EF
:105F5000C0470020436F756C64206E6F74207072B0
:105F60006F7465637420536F667444657669636506
:105F700020616E64206170706C69636174696F6E1A
:105F80002C20307825782E0004C8070070B5084D05
:105F900004460E46686805F075FE002C06D03246B1
:105FA00021466868BDE8704005F05EBE70BD000027
:105FB000F42A00200348D0F804050349097B00EBCC
:105FC0000160704700400240F42A002030B50A0505
:105FD00002D1B0F5FE2F01D9072030BD094C22684F
:105FE000082A01D3042030BD074B03EB0213C3F88A
:105FF0000008C3F804180220C3F80808521C002047
:10600000226030BDF02A002000E001402DE9F0417F
:106010003A483B49384E401AC508042000EB054079
:106020000027044637A102F0AFFDB06801280ED06A
:10603000A52813D0AA2818D0AC281ED0032000EB26
:10604000054039A102F0A0FD0020BDE8F081204606
:106050003CA102F099FDFDF761FC0CE020463CA15B
:1060600002F092FD04F038FF0DE020463BA102F063
:106070008BFDFDF7E3FE024607E020463AA102F061
:1060800083FD04F0F7FF024601271D491B4B012049
:10609000591AC90800EB014522B1284636A1B36858
:1060A00002F07DFD304600F0D1FBDFF800810021D9
:1060B00088F800103E4801F017FB064698F80000EB
:1060C00020B93C4940F2A510FDF7AEFE2EB128469E
:1060D00039A102F059FD0320B7E70120002FB4D009
:1060E00005492439096A0129AFD12046394902F00E
:1060F0004BFD0220A9E70000E447002088D80700F4
:1061000038D80700456E746572206E72665F626FE4
:106110006F746C6F616465725F66775F61637469E9
:1061200076617465000000004E6F206669726D77BD
:1061300061726520746F2061637469766174652E85
:106140000000000056616C6964204170700000001E
:1061500056616C69642053440000000056616C690C
:106160006420424C0000000056616C696420534476
:10617000202B20424C0000004163746976617469F1
:106180006F6E206661696C6564207769746820654C
:1061900072726F72202564202862616E6B20636FBB
:1061A00064653A203078257829000000242B0020EF
:1061B00069520700A0C80700436F756C64206E6FBA
:1061C000742077726974652073657474696E67737F
:1061D0002E00000038C907002DE9F041044641486F
:1061E0004149401AC108042000EB014005463FA187
:1061F00002F0CAFC434F00207C6001F007F9002840
:1062000059D1FFF703FF384A364B01219A1AD208B9
:106210004FF0000801EB024420B101281BD00228F6
:1062200049D105E04FF47016FEF72AFE10B93FE0A1
:106230004FF4A02600F0CEF8334A20211820FDF7B5
:106240004DFD08B1FDF71EFC3048016801F0F90171
:10625000B12904D007E00120FEF740FC3CE00168D2
:1062600001F04E0101602A48816D012907D1C0F873
:106270005880002001F01EFA08B1FDF703FC00F081
:106280009DFEC0B923493046FFF780FE224800F04A
:1062900049FE80B9284621A102F076FC00F086F87C
:1062A000FDF7FCFC02F000FB0028F7D141DFF5E729
:1062B00001F032F810B10320BDE8F08187F80080CA
:1062C0001A4801F09DF8387820B919A140F206204B
:1062D000FDF7AAFDFFF744FD204625A102F054FC7E
:1062E000E9E7000088D8070038D80700496E206E1B
:1062F00072665F626F6F746C6F616465725F696E06
:1063000069740000E82A0020082C00201C050040C9
:10631000C04700203555070061500700456E746581
:1063200072206D61696E206C6F6F70005D520700A6
:106330002E2E5C2E2E5C2E2E5C2E2E5C2E2E5C6362
:106340006F6D706F6E656E74735C6C696272617292
:106350006965735C626F6F746C6F616465725C6EAB
:1063600072665F626F6F746C6F616465722E63003A
:10637000556E726561636861626C650010B540F6C8
:10638000F8700168491C02D1074902F0F7FD40F698
:10639000FC700168491C05D1BDE810404FF4FC2198
:1063A00002F0ECBD10BD00000020070010B503F0A6
:1063B0004FF9002803D0BDE8104005F0C5BD10BD61
:1063C000034A93680A4601469860184605F04CBC9B
:1063D000F42A00202DE9F0411A4E307800282ED101
:1063E00003F036F91849194A0127891AC908032206
:1063F00002EB014500281DD01548046828462246B6
:1064000014A102F0C5FBA4F54864962C00DA96248A
:1064100005F09AFD2846224615A102F0B9FB214954
:106420002046FFF7CDFF4FF0E0214FF48030C1F858
:10643000000103E028461CA102F0A6FB3770BDE86E
:10644000F0810000252B002038D8070038D807003D
:106450000405014057445420656E61626C656420F8
:106460004352563A2564207469636B730000000040
:106470005374617274696E6720612074696D65720E
:1064800020282564207469636B732920666F72204D
:1064900066656564696E67207761746368646F67B9
:1064A0002E00000085BF0700574454206973206EFA
:1064B0006F7420656E61626C65640000406880687E
:1064C000004710B542680830527900F0F1F800201A
:1064D00010BD2DE9F04399B01C4690460D46084684
:1064E000DDF88090FFF7EAFF6E6807467079A042FA
:1064F00000D804462246414611A800F015F97279E9
:10650000494601A800F0D4F801AB224611A905F1D3
:1065100008000097FCF758F918B1002019B0BDE841
:10652000F08348F24250F9E770B516460C4605462E
:1065300000F0E2F800280ED1AA791946304600F0A2
:10654000E8F8002807D131462046FFF7BAFF0028B7
:1065500001D10149216070BD7052464D2DE9F843CB
:106560000C46DDE908578146984616460D492046F7
:1065700000F0B6F8002810D1606839464079420032
:10658000284600F0C6F8002807D146B143463246F7
:10659000214648460095FFF79CFFBDE8F88348F286
:1065A0001050FAE77052464D2DE9F0411D46DDE9E5
:1065B00006871646044600F02DF800280DD12A461D
:1065C0003146204600F03CF8002806D13A464146C4
:1065D0002046BDE8F04100F002B8BDE8F08170B59A
:1065E00015460E46044605F09FFC002807D13EB133
:1065F00060682968C268914205D248F2145070BDA3
:1066000048F2135070BD83682A4631462046BDE8E3
:106610007040184710B550B161B141600968044637
:106620008847002802D105482060002010BD48F2AC
:10663000015010BD48F2105010BD00006E52464887
:1066400070B515460E46044605F06EFC00280BD1C9
:1066500046B155B160682A46314643682046BDE8D8
:106660007040184748F2105070BD002070BD000007
:106670002DE9F0410B480C4D0C4F401BC608012082
:106680003870002406E000BF55F834008047002829
:1066900005D1641CB442F7D3022038700020BDE855
:1066A000F08100000000000000000000262B002008
:1066B00070B514460D46064600F036F82919301913
:1066C0002246BDE8704000F02FB870B50C46054674
:1066D00000F064F828192146BDE8704000F05EB86B
:1066E00028B10068884205D048F24050704748F20F
:1066F000105070470020704728B139B10022C1E91D
:1067000000201046704748F21050704748F213506E
:10671000704720B1914205D048F21150704748F2BD
:10672000105070470020704770B516460C460500A3
:1067300003D10AA14520FDF777FB1CB907A146202C
:10674000FDF772FBA919491E04E000BF14F8010B04
:1067500001F80109A942F9D270BD00002E2E5C2E6D
:106760002E5C2E2E5C2E2E5C2E2E5C636F6D706F59
:106770006E656E74735C6C69627261726965735C7C
:1067800063727970746F5C6E72665F637279707435
:106790006F5F7368617265642E63000070B50D46AB
:1067A000040003D107A13320FDF73EFB6019401E12
:1067B00005E02178027804F8012B00F80119A042C5
:1067C000F7D270BD2E2E5C2E2E5C2E2E5C2E2E5CF3
:1067D0002E2E5C636F6D706F6E656E74735C6C698A
:1067E000627261726965735C63727970746F5C6EFA
:1067F00072665F63727970746F5F736861726564EB
:106800002E6300004FF44050074A4168914207D17F
:106810008068411EC1F30B01401A00F6FF707047FB
:106820004FF4805070470000DBE5B15100B5FFF731
:10683000E9FF054989690A18401E0844C0F30B00A6
:10684000101A00F6FF7000BDC04700200021016053
:10685000416081600148016370470000C04700202B
:106860002DE9FF4F8B466948694981B0401AC1083C
:10687000042000EB0144009166A1204602F084F957
:1068800020466CA1019A02F083F9BBF1000F01D000
:106890006EA200E06FA2204670A102F079F9039881
:1068A00008B16AA200E06BA2204671A102F070F963
:1068B000049808B165A200E066A2204670A102F02B
:1068C00067F94FF4405041687348814201D15FA29B
:1068D00000E060A2204671A102F05AF9204673A19F
:1068E00002F052F9754D204675A1AB692A6A02F093
:1068F00056F920467AA16B6AEA6A02F050F94FF025
:106900000009DFF8FCA10CE0012650B1012812D0EB
:10691000B9F1020F1ED07B49AC20FDF785FA0020AB
:106920001AE0FFF783FF8046039888B16348006A46
:1069300001280BD00CE0FFF765FF8046049828B9CA
:106940004FF4405041685448814201D0012604E090
:10695000002602E04FF480508046D04503D96949B3
:10696000B120FDF761FA68490198A1EB0801A1F592
:106970000051814201D2012700E0002747EA0B05C0
:1069800020464A4661A102F003F92046424662A130
:1069900002F0FEF80FB12DA200E02EA2204664A165
:1069A00002F0F6F80EB129A200E02AA2204666A164
:1069B00002F0EEF80DB125A200E026A2204667A164
:1069C00002F0E6F8B54308D0B9F1020F05D209F19B
:1069D0000100C0B28146022896D957B10098022121
:1069E00001EB004062A102F0CFF8042005B0BDE841
:1069F000F08FB9F1000F07D0204668A102F0C4F86B
:106A00002E481830FFF722FF0020EFE788D8070054
:106A100038D80700456E746572206E72665F6466D2
:106A2000755F63616368655F707265706172652828
:106A30002900000072657175697265645F73697A17
:106A4000653A20307825782E000000007472756554
:106A50000000000066616C736500000073696E677A
:106A60006C655F62616E6B3A2025732E000000003A
:106A70006B6565705F6170703A2025732E000000B1
:106A80006B6565705F736F66746465766963653A9C
:106A90002025732E00000000DBE5B15153445F5008
:106AA000524553454E543A2025732E0042616E6B79
:106AB00020636F6E74656E74733A0000C0470020E7
:106AC00042616E6B203020636F64653A2030782518
:106AD0003032783A2053697A653A20307825780048
:106AE00042616E6B203120636F64653A20307825F7
:106AF0003032783A2053697A653A20307825780028
:106B0000000007007CCC0700002007007061737351
:106B10003A2025642E00000063616368655F61644C
:106B200064726573733A20307825782E0000000077
:106B300063616368655F746F6F5F736D616C6C3AFE
:106B40002025732E000000006B6565705F6669721A
:106B50006D776172653A2025732E000064656C655F
:106B600074655F6D6F72653A2025732E000000001A
:106B700041626F7274696E672E2043616E6E6F742E
:106B800020666974206E6577206669726D77617220
:106B900065206F6E2064657669636500496E766175
:106BA0006C69646174696E67206170702E0000000A
:106BB00070B50C46050004D121494FF4AC70FDF7C7
:106BC00033F924B91E4940F25910FDF72DF91D483B
:106BD0001D4B2978C01A0422C00802EB0040092985
:106BE00027D2DFE801F02605260B15261B260F000D
:106BF00021462846BDE8704002F032BD13A101F0E5
:106C0000C3FF11E021462846BDE8704002F0CCBD2C
:106C100021462846BDE8704002F064BD14A101F091
:106C2000B3FF4FF40070E0602046BDE87040FDF710
:106C3000FFBFBDE8704002494FF4BC70FDF7F4B8E7
:106C4000DCCA070050D8070038D8070048616E64D6
:106C50006C65204E52465F4446555F4F505F43522D
:106C6000435F4745542028636F6D6D616E64290052
:106C700048616E646C65204E52465F4446555F4FD6
:106C8000505F4F424A4543545F53454C454354205F
:106C900028636F6D6D616E642900000070B50E464B
:106CA000040004D11B4940F27520FDF7BDF826B958
:106CB000184940F27620FDF7B7F820780125092819
:106CC00020D2DFE800F01F051F0F141F1A1F0A0053
:106CD0003146204602F04EFE19E03146204603F0D0
:106CE0009FF814E03146204602F006FE0FE03146E0
:106CF000204602F049FF054609E03146204603F0F0
:106D000043F804E0034940F29720FDF78DF8284648
:106D100070BD0000DCCA07002DE9F843134C07469C
:106D20000D4620680090124812499046401AC60845
:106D3000042000EB06402B463A460FA101F037FF36
:106D400043462A4639461C4801F040FB050009D05D
:106D5000022000EB06402A4618A101F019FF284640
:106D6000BDE8F8832068401C2060F8E7442B002031
:106D700048D8070038D807006E72665F6673746F74
:106D8000726167655F657261736528616464723DF5
:106D9000307825702C206C656E3D2564207061670D
:106DA0006573292C2071756575652075736167653C
:106DB0003A20256400000000F42B00206E72665F0C
:106DC0006673746F726167655F65726173652829A8
:106DD000206661696C6564207769746820657272E9
:106DE0006F7220307825782E000000000C490D4A83
:106DF00010B5891AC908042202EB01420028104686
:106E000004D009A101F0C0FE114903E011A101F075
:106E1000BBFE1A49BDE810400022194801F036BBFC
:106E200048D8070038D80700496E697469616C69F1
:106E30007A696E67206E72665F6673746F726167DF
:106E4000655F7364206261636B656E642E00000091
:106E500034C40700496E697469616C697A696E6748
:106E6000206E72665F6673746F726167655F6E76BF
:106E70006D63206261636B656E642E0004C407005D
:106E8000F42B00202DE9FC47154C80460F46206866
:106E90001549CDE9002013489946401AC608154601
:106EA000042000EB06403B464246104901F088FEB4
:106EB0002B463A4641460E48CDF8009001F0AEFB15
:106EC000050009D0022000EB06402A4609A101F086
:106ED0005FFE2846BDE8FC872068401C2060F8E77C
:106EE000442B002048D8070038D8070024CA0700E0
:106EF000F42B00206E72665F6673746F7261676553
:106F00005F77726974652829206661696C65642001
:106F100077697468206572726F7220307825782ED8
:106F20000000000070B51149086011481149401A6D
:106F3000C508032000EB05400FA101F025FE00204D
:106F4000FEF7B2F8114800F041FC040008D001201F
:106F500000EB054022460EA101F01AFE204670BD4E
:106F6000BDE87040094800F0A7B80000282B0020B9
:106F700088D8070038D80700456E746572696E6757
:106F800020444655206D6F64652E0000A95007000F
:106F9000436F756C64206E6F7420696E6974616CE8
:106FA000697A6520444655207472616E73706F7201
:106FB000743A2030782530387800000006480749B8
:106FC00010B5401AC008042101EB004004A101F0F3
:106FD000DBFD002010BD000088D8070038D807006E
:106FE000696E207765616B206E72665F6466755F9F
:106FF000696E69745F757365720000001FB589085A
:10700000002201AB009283E80700684618DF04B055
:1070100010BD00001FB5044B0FCB8DE80F00684674
:1070200018DF04B010BD0000A8C307004FF4805063
:10703000410408600020704770B50E460178134C7B
:10704000062901D0012901D1017C21702178012577
:10705000012911D0022913D00D480E49401AC00849
:10706000012101EB00400CA101F08EFD00202070F9
:1070700005207070284670BD3146FFF799FDF9E78D
:107080003146FFF70BFE0546F4E700004C2B0020CD
:1070900050D8070038D80700496E76616C696420C3
:1070A0006F626A656374207479706520696E2072FE
:1070B0006571756573742E0010B5040011D0012040
:1070C000FFF794FE00280BD100F0EEFC00F0CEFD9F
:1070D00048B10949081F00F057FD012803D00320DB
:1070E00010BD072010BD04480838C4600020FEF71A
:1070F000AFF8002010BD0000542B002010B58168AF
:1071000089B10A4A1821FCF779FD040009D0084822
:107110000849401AC008022101EB004006A101F015
:1071200033FD204610BD072010BD0000557107003B
:1071300050D8070038D807005363686564756C65DC
:10714000722072616E206F7574206F66207370619B
:1071500063652100AFF3008070B50546806886B096
:1071600020B9284940F2CF20FCF75EFE18222649BC
:107170006846FBF757F928788DF800002348244B20
:107180002A78181A0421C008224E01EB00440D2A67
:107190001CD2DFE802F01B140714141B141B141B71
:1071A0001B1B0C0020461CA101F0EEFC17E0204642
:1071B00022A101F0E9FCF168072088470FE0694649
:1071C0002846FFF739FF50B906B070BD032101EB27
:1071D000004020A101F0DCFC02208DF801009DF8A8
:1071E0000120204623A101F0D3FCD5E90112684615
:1071F00090479DF801000128E6D0F16805208847F6
:10720000E2E70000DCCA0700D0C3070038D8070057
:1072100050D807004C2B002048616E646C65204EEE
:1072200052465F4446555F4F505F52454345495073
:10723000545F4E4F5449465F5345540048616E6455
:107240006C65204E52465F4446555F4F505F414249
:107250004F525400496E76616C6964206F70636FA1
:1072600064652072656365697665643A20307825C7
:10727000782E0000526571756573742068616E64C4
:107280006C696E6720636F6D706C6574652E20523B
:107290006573756C743A20307825780038B10549EB
:1072A00001600549416001210172002070470E20F4
:1072B00070470000BD720700F572070010B50C00A2
:1072C00001464FF0110007D02278052A05D2DFE8E9
:1072D00002F00F050D0F0F000E2010BD084600F044
:1072E00073F80028F9D10221217010BD112010BDC2
:1072F000082010BD0246082041B10B78022B04D1B2
:10730000022A05D0032A00D1112070470E207047B1
:10731000002003220A70704770B510480024D0F88E
:107320002413491C03D1D0F86403401C13D00C482B
:107330000C49401AC008042101EB00400AA101F0E9
:1073400023FC4FF4FE25284601F000FEC922034924
:10735000284601F02BFE204670BD0000C0470020EB
:1073600060D8070038D8070045726173696E6720DE
:1073700073657474696E67732070616765206164FA
:10738000646974696F6E616C20646174612E0000C1
:1073900010B528B11C220349FBF744F8002010BDAA
:1073A0000E2010BD64F3070010B5064C0022182112
:1073B000201DFDF74FFC2168814201D1012010BD45
:1073C000002010BD64F3070070B50C4D0400D5F823
:1073D000640305F5597503D0401C03D0082070BD27
:1073E0000E2070BD00221821201DFDF733FC206007
:1073F00007222146284629DF70BD000000F0070063
:10740000014903F03FBF000000F0070070B50546DA
:1074100012481349401AC408042000EB044011A18B
:1074200001F0B2FB2846FFF7E1FC02004FF001003B
:1074300000EB044402D0204613A108E000F06CF8F1
:10744000002000F051F9020005D0204619A101F0FA
:107450009FFB032070BD002070BD000058D80700BE
:1074600038D8070043616C6C696E67206E72665F86
:107470006466755F73657474696E67735F696E695E
:107480007428292E2E2E00006E72665F6466755F6A
:10749000666C6173685F696E69742829206661692A
:1074A0006C65642077697468206572726F723A2027
:1074B000257800006E72665F6466755F736574742C
:1074C000696E67735F77726974655F616E645F622E
:1074D00061636B75702829206661696C656420772B
:1074E000697468206572726F723A20257800000016
:1074F00010B5FF224FF400710648FAF7A5FF0548C2
:1075000020212438FAF7A7FF024900205C390863DC
:1075100010BD00001C4800202DE9F05F4048FDF739
:10752000B7FB404E074634682046FDF7B1FB4FF0ED
:10753000000A58B16068012806D02046FDF73CFAE1
:10754000D4F85C12884201D1012400E000243648BE
:107550003649DFF8DC80401AC00803214FF00209E9
:107560004FF4607B01EB0045F7B1042101EB0040D3
:10757000074630A101F008FB5A4629494046FAF770
:1075800051FFDCB1384631A101F0FEFA36684446BD
:107590005422311D201DFAF745FF4FF4327206F1D7
:1075A0005C0104F15C0007E06CB32846324901F04D
:1075B000EBFA5A461E483168FAF734FFD8F804004F
:1075C000444601281DD128462CA101F0DDFA364998
:1075D000402201F5E470FAF725FF33491C224031BF
:1075E00001F5E470FAF71EFF84F860A2012184F827
:1075F000A1122E4884F8E2A2E169C0F82210C4F872
:107600000490BDE8F09F4C4609EB0040284901F08A
:10761000BBFA59460648FAF71EFFC8F80440F0E7DF
:1076200000F007005C2B002058D8070038D807006E
:10763000C04700205573696E672073657474696E66
:10764000677320706167652E00000000436F7079DA
:10765000696E6720666F7262696464656E2070612E
:107660007274732066726F6D206261636B75702037
:10767000706167652E0000008CCB07004F6C6420A2
:1076800073657474696E67732070616765206465E3
:107690007465637465642E20557067726164696EE9
:1076A0006720696E666F2E001C490020404A00204A
:1076B00028CB070070B50546094803F04FFE084C7B
:1076C00020602046FDF778F9C4F85C02A4F5E06379
:1076D0002A462146BDE87040024803F045BE00003E
:1076E000C047002000F0070070B505460020FFF7F6
:1076F000E1FF040003D10349284603F0C3FD2046FF
:1077000070BD0000C04700204FF48050704700005B
:107710002DE9F0471449DFF854808146A1EB0800B9
:10772000C708134813490026401AC108042000EB7B
:10773000014005463A4610A101F02AFA00240EE065
:1077400008EBC400416848468847060006D0284632
:107750003346224612A101F022FA02E0641CBC4228
:10776000EED33046BDE8F08728D8070020D80700C0
:1077700088D8070038D807005368757474696E6735
:1077800020646F776E207472616E73706F727473A1
:107790002028666F756E643A202564290000000079
:1077A0004661696C656420746F2073687574646FDA
:1077B000776E207472616E73706F72742025642C02
:1077C000206572726F722025640000002DE9F04779
:1077D0001449DFF854808146A1EB0800C70813481C
:1077E00013490026401AC108042000EB0140054659
:1077F0003A4610A101F0CCF900240DE058F83410FD
:1078000048468847060006D028463346224612A13D
:1078100001F0C5F902E0641CBC42EFD33046BDE87C
:10782000F087000028D8070020D8070088D8070074
:1078300038D80700496E697469616C697A696E6746
:10784000207472616E73706F7274732028666F7526
:107850006E643A20256429004661696C6564207471
:107860006F20696E697469616C697A6520747261F0
:107870006E73706F72742025642C206572726F7243
:1078800020256400012203F0B3B8000038B5144687
:1078900002780B46FAB1012A09D0022A1DD0032A28
:1078A00023D0174940F2D930FCF7BEFA25E0D0F8D2
:1078B0000150002221461846FDF7CCF9A8420AD013
:1078C000104811490122401AC008042101EB004070
:1078D0000EA101F05DF9012038BD01B02246BDE8DE
:1078E00030400023401C00F023B8411C40220020FF
:1078F000009400F017FA0128EED0002038BD0000F7
:10790000BCCE070068D8070038D807004352432090
:10791000636865636B206F662061707020666169C3
:107920006C65642E2052657475726E2025640000AB
:107930002DE9F043A9B007462020894628901C462F
:1079400090460125782102A8FAF785FDFDF7B0F9E8
:107950002CB12022394620A8FEF7E6FE20AF2448AD
:1079600024494346401AC608042000EB064004465A
:107970004A4621A101F013F928A92C48CDE90001BC
:1079800043464A462A4902A8FEF70EFE020006D0E8
:10799000012000EB064027A101F0FAF822E02022A6
:1079A00039462248FAF769FDE8B1022000EB0640AB
:1079B0002DA101F0E9F8204632A101F0E5F82046BA
:1079C0002022394601F08AF8204633A101F0DCF884
:1079D00020462022154901F081F800BF00F064FF25
:1079E0000028FBD1002529B02846BDE8F08300001F
:1079F00068D8070038D80700486173682076657238
:107A0000696669636174696F6E2E20737461727444
:107A100020616464726573733A20307825782C2075
:107A200073697A653A20307825780000144F002079
:107A3000B8C00700436F756C64206E6F7420727558
:107A40006E20686173682076657269666963617427
:107A5000696F6E20286572725F636F64652030788D
:107A60002578292E00000000486173682076657231
:107A7000696669636174696F6E206661696C6564CB
:107A80002E000000457870656374656420465720B9
:107A9000686173683A00000041637475616C204648
:107AA0005720686173683A0010B50648064C806B31
:107AB00020B103F07BFF08B1012000E0002020701E
:107AC00010BD0000C0470020602B00202DE9F041D0
:107AD000144C07460D46E06BA26B012641199142FA
:107AE0000BD911481149401AC008012101EB00408F
:107AF0000FA101F049F8032610E00A492A465C313B
:107B000008443946FAF78EFCE06B064A2844E063E5
:107B1000403229463846FDF79DF820643046BDE8DE
:107B2000F0810000C047002068D8070038D807005F
:107B3000496E697420636F6D6D616E64206C617253
:107B4000676572207468616E20657870656374651E
:107B5000642E000070B504004FF0010504D0B4F5A8
:107B6000007F03D9042508E0032506E0044900202E
:107B70000870FFF7BDFC03488463284670BD000011
:107B8000602B0020C04700202DE9F0410646244824
:107B90000F46254BD0E90E1222484FF00108C01ABB
:107BA000C00808EB00448A4205D020461FA100F01F
:107BB000EBFF082430E0244D287840B1FEF736FE74
:107BC00030603946E86804F043F9044624E003F0E5
:107BD000EDFEE0B100F050F804460020306038605F
:107BE000012C0ED13946E86804F032F90446012828
:107BF00007D132463968E86804F0E6F804460128FF
:107C000002D0FFF775FC07E085F8008004E020460D
:107C10000EA100F0B9FF05242046BDE8F081000068
:107C2000C047002068D8070038D80700457865634A
:107C30007574652077697468206661756C74792045
:107C40006F66667365740000602B00204661696C86
:107C5000656420746F206465636F646520696E6974
:107C600074207061636B6574000000000148007847
:107C700070470000602B0020F8B51C4C251D00202B
:107C800094F86C31014602463BB194F8D802B4F83E
:107C9000DA2204F5B87504F53771154CA368009322
:107CA000636800F03FF80646012805D1281D00F062
:107CB00043F90646012816D00E480F49401AC50858
:107CC000022000EB05400DA100F05EFF042000EB58
:107CD000054510A1284600F057FF2089616882B24F
:107CE000284600F0FBFE3046F8BD0000404B002067
:107CF000602B002068D8070038D8070050726576DE
:107D0000616C69646174696F6E206661696C656439
:107D10002E000000496E697420636F6D6D616E64A2
:107D20003A0000002DE9F047A2B080462020DDF89F
:107D3000A8900F4620909A461646782102A8FAF796
:107D40008AFB00202190FCF7B3FF40484049401ACD
:107D5000C508032000EB054004463EA100F014FFD7
:107D600057B1B8F1000F20460ED044A100F00CFF2F
:107D7000162022B0BDE8F087022000EB054045A1A7
:107D800000F002FF1320F4E74A4647A100F000FF8D
:107D900020A94C48CDE900014B4652464A4902A869
:107DA000FEF702FC08B9402E01D00A20E1E7454861
:107DB000324639464038FAF735FB204643A100F0F9
:107DC000E3FE404820214038FEF77FFC3D4840213B
:107DD0004038CDE90001A0F148013A4A21A8209B92
:107DE000FEF7BCFB02002BD0012000EB05403CA1BC
:107DF00000F0CEFE042000EB054442A1204600F036
:107E0000C3FE304920464022403900F067FE20463C
:107E10003FA100F0B9FE20982A4982B2204600F026
:107E20005DFE20463CA100F0AFFE204640223D49C9
:107E300000F054FE00F038FD0028FBD1052098E743
:107E4000204639A100F0A0FE012092E768D8070083
:107E500038D807005369676E617475726520726562
:107E60007175697265642E20436865636B696E671E
:107E7000207369676E61747572652E00496E766154
:107E80006C6964207369676E6174757265207479BA
:107E9000706500004E6F207369676E61747572655E
:107EA00020666F756E642E0043616C63756C61743F
:107EB000696E67206861736820286C656E3A2025BA
:107EC00064290000F44E0020B8C0070056657269AE
:107ED0006679207369676E617475726500000000D1
:107EE0005369676E6174757265206661696C65645B
:107EF00020286572725F636F64653A203078257858
:107F0000290000005369676E61747572653A00005C
:107F1000486173683A0000005075626C6963204BD9
:107F200065793A0058C00700496D6167652076653C
:107F300072696669656400002DE9F04104004FF044
:107F4000010603D13349C420FBF76EFF3248334AA0
:107F500094F85410801AC008012202EB004541B188
:107F600094F8550040B1012806D0022804D0032817
:107F700002D028462AA147E01CB92649A320FBF7D6
:107F800053FF94F86E00032805D028462AA100F07C
:107F9000FBFD14263BE094F8920018B194F893008E
:107FA000002834D1207A78B11C4A1B4B02209A1A3F
:107FB000D208E16800EB0247342908D0384623A1F3
:107FC00000F0E2FD112622E0284625A11CE0204613
:107FD00003F0BEF830B1207880B12046FDF760F99B
:107FE00030B114E0384622A100F0CEFD12260EE09A
:107FF000384623A100F0C8FD102608E094F855008B
:10800000012804D0284623A100F0BEFD0F263046EB
:10801000BDE8F08104CF070070D8070038D807000A
:10802000496E76616C6964206669726D776172650C
:1080300020747970652E0000496E76616C69642049
:108040006861736820747970652E00004661756CF4
:1080500074792048572076657273696F6E2E000020
:108060004E6F2048572076657273696F6E2E000040
:10807000534420726571206E6F74206D65742E00FC
:1080800046572076657273696F6E20746F6F206C2F
:108090006F772E0046572076657273696F6E206D7C
:1080A000697373696E672E000FB438B5040003D18D
:1080B00010A14220FBF7B8FE606918B90DA143205A
:1080C000FBF7B2FE206818B90AA14420FBF7ACFE0A
:1080D000606818B907A14520FBF7A6FE059900299D
:1080E00005D006A800906A46204600F045F838BC46
:1080F0005DF814FB2E2E5C2E2E5C2E2E5C2E2E5C3C
:108100002E2E5C65787465726E616C5C6670726947
:108110006E74665C6E72665F667072696E74662EEF
:108120006300000010B5040003D107A13120FBF764
:108130007BFEA268002A05D0D4E904032168984791
:108140000020A06010BD00002E2E5C2E2E5C2E2E76
:108150005C2E2E5C2E2E5C65787465726E616C5C94
:10816000667072696E74665C6E72665F6670726964
:108170006E74662E630000002DE9FC4791460C46A4
:108180005FEA000804D183A140F25220FBF74CFEC5
:10819000D8F8140020B97FA14FF41570FBF744FE06
:1081A000D8F8000020B97BA140F25520FBF73CFE37
:1081B000D8F8040020B977A140F25620FBF734FE2E
:1081C000002C76D014F8011B39B125290ED0404679
:1081D000FCF70AFD20780028F4D198F80C0000285C
:1081E00067D04046BDE8FC47FFF79CBF0020012256
:1081F00021782B291BD02D2902D0302908D102E06B
:1082000040F0010001E040F00200641C002AEFD1C0
:1082100000252A290ED02178A1F130020A2A11D294
:1082200005EB850201EB4205641C303DF1E740F0AF
:108230000400EAE7D9F800100B1DC9F800300968FE
:10824000641C0D44217800232E290BD114F8011F42
:10825000A1F130020A2A05D203EB830201EB4203AB
:10826000303BF3E76C290DD068290BD0692921D068
:108270000BDC252918D0582931D063290ED0642968
:1082800015D117E014F8011FECE7702969D07329A4
:1082900032D075291BD0782909D120E0D9F8000007
:1082A000011DC9F8001001784046FCF79DFC641CD4
:1082B00090E76CE0D9F800100A1DC9F800200968A1
:1082C000CDE900500A224046FDF774F9EFE7D9F8EE
:1082D00000100A1DC9F8002009680A2206E0D9F832
:1082E00000100A1DC9F8002009681022CDE90050CD
:1082F000404603F00FFDDAE7D9F8001000270A1D09
:10830000C9F800200E68C00705D112E04046761C6F
:108310007F1CFCF769FC31780029F7D104E02021AB
:1083200040466D1EFCF760FCBD42C0D9002DF6D161
:10833000BDE74EB13046FAF799F8074604E0202130
:1083400040466D1EFCF750FCBD4206D9002DF6D10B
:1083500003E04046761CFCF747FC31780029F8D151
:10836000A5E7D9F80000011DC9F800100568302103
:108370004046FCF739FC78214046FCF735FC0820E4
:108380000021CDE90001034610222946B0E7BDE8EF
:10839000FC8700002E2E5C2E2E5C2E2E5C2E2E5C7A
:1083A0002E2E5C65787465726E616C5C66707269A5
:1083B0006E74665C6E72665F667072696E74665F1C
:1083C000666F726D61742E63000000002DE9F0414C
:1083D0001E4615460F46040003D11DA19E20FBF743
:1083E00023FD206818B91AA19F20FBF71DFD1DB9B8
:1083F00017A1A020FBF718FD39462046FBF712FA1B
:1084000040B939462046FBF70DFA18B910A1A32050
:10841000FBF70AFD60683946026820466A43FBF7AD
:108420000AFA58B960683946026820466A43FBF781
:1084300002FA18B906A1A520FBF7F6FC206833461E
:108440002A46D0F810C039462046BDE8F0416047C2
:108450002E2E5C2E2E5C2E2E5C2E2E5C2E2E5C6321
:108460006F6D706F6E656E74735C6C696272617251
:108470006965735C6673746F726167655C6E726662
:108480005F6673746F726167652E630070B5164620
:108490000C46050003D108A15520FBF7C5FC1CB90B
:1084A00005A15620FBF7C0FC2C6031462846226807
:1084B000BDE87040104700002E2E5C2E2E5C2E2E44
:1084C0005C2E2E5C2E2E5C636F6D706F6E656E740D
:1084D000735C6C69627261726965735C6673746FF8
:1084E000726167655C6E72665F6673746F726167F6
:1084F000652E63002DE9F04128B1016819B1C96901
:10850000BDE8F04108470D4D0D480024461B1427D7
:108510000DE000BF04EB840005EB8000016829B189
:10852000C969884710B10120BDE8F081641CB6FB21
:10853000F7F0A042EED80020F6E70000F42B002070
:10854000082C0020044801214174007A08B1002061
:1085500070470120704700002C510020012801D0F5
:10856000032808D10449002201284A7400D00020C1
:10857000087402F0E3BB70472C51002070B501462F
:10858000022801D0032943D1224C207A00283FD071
:10859000012831D002282FD11F480023022900686A
:1085A00002D0032928D119E0E360027912B1012A2F
:1085B00022D10BE0D0E90565721B142A00D31422E6
:1085C0002A4482614569AA420ED015E00169491C1E
:1085D0000161426991420FD1237213E0E268521C9B
:1085E000E260082A08D9E360237202290AD00D212B
:1085F000FCF7F5FD02F098FB607C28B1BDE8704007
:1086000000F0FCBE0021F3E7BDE8704002F096BB2D
:1086100070BD00002C510020842B00202DE9F84370
:108620001D46089F16468846040003D12AA18820CB
:10863000FBF7FAFB1EB928A18920FBF7F5FB2068A0
:1086400018B925A18A20FBF7EFFB1DB922A18B20C9
:10865000FBF7EAFB60684068B5FBF0F100FB1151E5
:1086600041B1B5FBF0F100FB115018B11AA18E20F9
:10867000FBF7DAFB4046FBF7CFF838B94046FBF78B
:10868000CBF818B914A19120FBF7CEFB3046FBF7CD
:10869000C3F838B93046FBF7BFF818B90EA19220DD
:1086A000FBF7C2FB2A4641462046FBF7C4F848B90F
:1086B0002A4641462046FBF7BEF818B906A193208A
:1086C000FBF7B2FB009720682B463246C76841464D
:1086D0002046B847BDE8F8832E2E5C2E2E5C2E2E49
:1086E0005C2E2E5C2E2E5C636F6D706F6E656E74EB
:1086F000735C6C69627261726965735C6673746FD6
:10870000726167655C6E72665F6673746F726167D3
:10871000652E630030B5134B014600201C692246CC
:108720000AE0D2681579854205D1401C0A28F6DB9B
:108730004FF0FF3030BD1268002AF2D1421CF9D050
:10874000CA6810711A693AB1D268CC68126822609E
:108750001A69D268116030BD1961C96800220A60C7
:1087600030BD0000D86200207047FAF7C9BE7047DC
:1087700008B5034A00924023024A00F005F808BDFC
:1087800035B2070040510020F0B595B01C461546A3
:108790000E4608461A9F00F069FB182109A8F9F750
:1087A0005AFE0E97CDE909540023082203A930464A
:1087B00000F072FB05980690BDF81000ADF81C00A3
:1087C000BDF81200ADF81E0000208DF821000399BD
:1087D000082501F00300012802D0022816D02FE05E
:1087E000C1F3C200C1F383178C0A8DF82000BA00D0
:1087F0002B460FA9304600F04FFB09A8009006ABAE
:108800003A460FA9204600F08DFA19E0C1F3C200E4
:108810008C0D8DF82000082C01D2274600E0082797
:108820002B463A460FA9304600F036FB3D44E41B88
:1088300009AB06AA39460FA800F0DAF9002CEAD1F4
:10884000304600F019FB15B0F0BD00000A4A0129BE
:1088500002EBC00007D0022907D0032907D0042962
:1088600007D000207047022070470420704700792D
:10887000704740797047000038D8070010B5FFF7FF
:1088800074FF04210648FFF745FF002803DA054975
:108890004120FBF7C9FA02490120C968487110BD9F
:1088A00028D8070090D307002DE9F04F8DB0FCF7D2
:1088B000B3F918B100200DB0BDE8F08F7C4E002058
:1088C000B061BFF34F8FA6F580547A49A06802903B
:1088D0000D684FF00009284004EB80000AE0B06901
:1088E00070B961680298814201D8A160E2E728402E
:1088F00004EB80000C3002A9FCF7AFFE0028EED19B
:10890000002009AAA046029901EA050308EB8303A7
:10891000491CDB6842F82030401C02910228F2D347
:10892000099800F00301022902D001294CD0A6E0E9
:10893000810D50228A46B2EB905F00D850210C4640
:1089400064F39F50099008315B4800F046FA070035
:1089500074D000F08BFA4B46082209A9384600F083
:10896000C9FA029909F1080B2940681A8000001D14
:10897000844222D9514D30B1C2B208EB8101201A94
:1089800091460C3104E02946E2B200259146284682
:10899000C4B25B46384600F0ADFA0BEB09032DB1CB
:1089A000224629464FEA070000F0A4FA02990AF18C
:1089B000030001EB9000029039E008EB81015B4677
:1089C000224638460C31EFE7C0F38311062900D365
:1089D000062161F389100990C0F38310801C810087
:1089E000354800F0FAF9070049D000F03FFA4B464D
:1089F000082209A9384600F07DFA09F10809002487
:108A00000FE002984B4600EA0501401C08EB81018B
:108A10000290042238460C3100F06CFA09F1040986
:108A2000641C0998C0F38310A042EAD837B13469B6
:108A3000B06978B1384600F01FFA34E01FE0E06812
:108A40004079012804D122682046394612689047AF
:108A5000E0680468002CF2D1384600F00DFA0020DE
:108A60008DF800006846FBF74FF9B06910B902991C
:108A7000C8F808109DF80000FBF792F913E034697C
:108A800005E02168204689688847E0680468002C72
:108A9000F7D10B480B49401AC008022101EB0040F6
:108AA00009A100F071F8FCF7B7F880F0010002E7C7
:108AB000D8620020982B0020BCD80700E452002088
:108AC00088D8070038D807004261636B656E64730D
:108AD00020666C7573686564000000002DE9F84F2E
:108AE0008146274FD01C15468A46800800226946D9
:108AF0003E68FCF71FF8DFF88C80B0B3009CA01C28
:108B0000009039683040091A8F003F1DBD4208EBC4
:108B1000800002D82A46514608E03A4651460C30B9
:108B2000F9F780FC1748EA1B0AEB07010C30F9F74C
:108B300079FC4FEA1947FCF7E3FA47EA0042601C68
:108B4000304008EB8000344008EB8401C260C86804
:108B50004FF6C07269F3C500904365F39F5020F053
:108B60000300801C20F00400C86098F8000001E0B9
:108B7000FFF79AFE0028FBD1FCF71BFEBDE8F88F3B
:108B8000982B0020D852002000231A4602F0D8BEAD
:108B900008B5012300926A4602F0D2FE08BD1CB55A
:108BA000CDE9002302236A4602F0CAFE1CBD3EB591
:108BB000069C8DE81C0003236A4602F0C1FE3EBD00
:108BC0007FB5DDE908458DE83C0004236A4602F0E4
:108BD000B7FE7FBD70B586B00DF1280C9CE8700023
:108BE0008DE87C0005236A4602F0AAFE06B070BD3F
:108BF0002DE9F0470E4680461C469246082940D88B
:108C000094F80C90002020731946104602F032F8B8
:108C10000025B54206D218F805201BA12046FFF713
:108C200043FA03E01AA12046FFF73EFA6D1C082D17
:108C3000EFD318A12046FFF737FA0025B54212D22C
:108C400018F805707E2F08D8F9F7E8FB0068C05DBA
:108C500010F03E0F01D03A4600E02E220EA1204631
:108C6000FFF722FA03E00DA12046FFF71DFA6D1C65
:108C7000082DE3D301222146504601F09BFE84F8E3
:108C80000C90BDE8F087000020253032780000000D
:108C9000202020007C000000256300002000000050
:108CA000064910B500200870054800F0E3F80028D8
:108CB00003D1044800F09CF9002010BDD8520020D8
:108CC000BCD80700A8C6070002480349401AC008DC
:108CD00070470000A8D8070038D8070013B56846C9
:108CE000FCF7A6FE08B100201CBD0248009950F810
:108CF00031001CBD38D8070070B50948012504694A
:108D0000A0F58050057007E0E068457121682046B5
:108D100049688847E0680468002CF5D170BD000000
:108D2000D86200202DE9FF4781460C9D00200C46AB
:108D30002F7B2873984616462946184601F09AFF5D
:108D4000072E42D2DFE806F004090F161F2A36006C
:108D500049462846FFF7A8F937E0494628462268E1
:108D6000FFF7A2F931E0D4E9002349462846FFF78E
:108D70009BF92AE0A0680090D4E9002349462846E0
:108D8000FFF792F921E0D4E90201CDE90001D4E92D
:108D9000002349462846FFF787F916E004F108004A
:108DA00007C88DE80700D4E9002349462846FFF7A5
:108DB0007BF90AE004F108000FC88DE80F00D4E940
:108DC000002349462846FFF76FF90022294640460E
:108DD00001F0F0FD2F73BDE8FF872DE9F041058A12
:108DE00080462D1F4819C01CB0FBF5F0C6B24046A6
:108DF000FCF7B0FE041E19D0002020710120607124
:108E0000E58000272546761EC4F800800BE040462A
:108E1000FCF7A0FE60B16179491C617128600546CC
:108E20007F1CC0F80080B742F1D32046BDE8F08136
:108E3000204600F002F80020F8E72DE9F0414579DE
:108E400001466B1E002201E00968521C9A42FBD3C6
:108E50000F680146002605E038460C68FCF7E0FE86
:108E60002146761CAE42F7D3BDE8F0810121001DFA
:108E7000FCF749BEFCF71CBF10B504460121001DDC
:108E8000FCF762FE10F0FF0F04D12046BDE8104051
:108E9000FFF7D3BF10BD00001CB514460122CDE979
:108EA000002401AAFCF756FD0198A04204D003A1BA
:108EB0004FF48070FAF7B8FF1CBD00002E2E5C2E18
:108EC0002E5C2E2E5C2E2E5C2E2E5C636F6D706FD2
:108ED0006E656E74735C6C69627261726965735CF5
:108EE0006D656D6F626A5C6E72665F6D656D6F62F7
:108EF0006A2E63001CB514460022CDE9002401AAA5
:108F0000FCF728FD0198A04203D002A1F620FAF751
:108F10008BFF1CBD2E2E5C2E2E5C2E2E5C2E2E5C0E
:108F20002E2E5C636F6D706F6E656E74735C6C6912
:108F3000627261726965735C6D656D6F626A5C6EA9
:108F400072665F6D656D6F626A2E63000949022269
:108F50000A60BFF36F8FBFF34F8F0A1D1060064882
:108F60000268002AFCD000200860BFF36F8FBFF3B7
:108F70004F8F704704E5014000E40140094A012396
:108F80001360BFF36F8FBFF34F8F01600648016816
:108F90000029FCD000201060BFF36F8FBFF34F8F0C
:108FA0007047000004E5014000E4014070B50E4C3C
:108FB00001232360BFF36F8FBFF34F8F00230B4D4F
:108FC00008E000BF51F8236040F823602E68002EAF
:108FD000FCD05B1C9342F5D300202060BFF36F8F61
:108FE000BFF34F8F70BD000004E5014000E4014075
:108FF0008268002191608268116182685161826893
:10900000D1608268516080680160704708B50022B5
:1090100042504058009008BD20B1034909680160E2
:10902000002070470E2070472CC707002DE9FE4333
:1090300007460E460846FFF7EFFF00287CD10024C4
:109040000094019406208DF800704FF00108ADF8EF
:10905000040002948DF8028069462020326869DF9E
:109060003649374A891AC908012202EB014530B155
:1090700000F09EFA024628463249FFF789FD009427
:109080008DF801808DF80240019402948DF8034020
:1090900069464020326869DF30B100F089FA024643
:1090A00028462949FFF774FD00948DF80070F720D9
:1090B000ADF802000194029469462320326869DF0A
:1090C00030B100F075FA024628462049FFF760FDEE
:1090D0000094019402948DF8008069460120326862
:1090E00069DF30B100F064FA024628461849FFF7FC
:1090F0004FFD4FF4B0600090019402946946A120A6
:10910000326869DF30B100F053FA0246284611494F
:10911000FFF73EFD0094019402948DF800406946EB
:10912000A020326869DF30B100F042FA02462846DA
:109130000949FFF72DFD0020BDE8FE8398D8070000
:1091400038D8070088D50700D0D507001CD60700FF
:10915000E8D4070034D5070094D407002DE9F04186
:109160000546076860DF804619491A482A68081AC8
:10917000C608BA4219D9022000EB064416A12046BF
:10918000FFF702FD20463A461FA12B68FFF707FDB7
:109190004FF08050D0F80C012968800200F1005097
:1091A000421A204625A1FFF7F3FCB8F100004FF06A
:1091B00001040AD000F0FCF9024604EB06402AA1A3
:1091C000FFF7E6FC4046BDE8F0812F480470F9E760
:1091D00098D8070038D80700496E737566666963CA
:1091E00069656E742052414D20616C6C6F636174CF
:1091F000656420666F722074686520536F667444DE
:1092000065766963652E00004368616E676520744A
:1092100068652052414D207374617274206C6F63D5
:109220006174696F6E2066726F6D203078257820CA
:10923000746F20307825782E000000004D61786929
:109240006D756D2052414D2073697A6520666F728D
:10925000206170706C69636174696F6E206973203E
:10926000307825782E00000073645F626C655F655E
:109270006E61626C6528292072657475726E656412
:109280002025732E00000000EF2B002030B5184879
:10929000ADF5017D0078002826D04FF4FA7400BFA8
:1092A000ADF8004280A9684661DF38B105281BD0BF
:1092B0000DF5017DBDE83040FAF7E4BB6D460D4980
:1092C0007DA800F0F1F809E07DA800F0D5F8D0E91C
:1092D0000021284690477DA800F024F97DA800F0E1
:1092E000CBF80028DCD0EFE70DF5017D30BD0000A4
:1092F000EF2B002030C70700F8B5134C2078C0B121
:109300000120A07001F060FF112814D0022001F0AC
:1093100077FF00258DF800506846FAF7F5FC11DF5D
:10932000064625709DF80000FAF73AFD2EB130464A
:10933000F8BD0820F8BD0020F8BDA57002F020FAA5
:10934000032001F05DFFF6E7EC2B00207CB5194C03
:10935000207808B108207CBD0120A070002001F019
:1093600033FF112819D0002001F04AFF12480026CF
:10937000006801908DF800606846FAF7C5FC0F4957
:1093800001A810DF05000AD0002020709DF8000021
:10939000FAF706FD2DB128467CBD00207CBD0120DA
:1093A000F3E7A670667002F04FFA012001F028FF83
:1093B000F3E70000EC2B0020C4C60700213A0700A9
:1093C0000EB50A49684600F06FF808E0684600F0FC
:1093D00047F8D0E900108847684600F0A3F86846CF
:1093E00000F03EF80028F1D10EBD0000E0C60700F5
:1093F0000148007870470000EC2B00200548817878
:1094000019B1007818B1FFF777BF08207047FFF750
:109410009DBF0000EC2B00201FB568464BDF30B12C
:10942000052819D004B0BDE81040FAF72BBB0B4952
:1094300001A800F039F809E001A800F029F8D0E906
:1094400000210098904701A800F06CF801A800F0F6
:109450001FF80028E1D0EFE71FBD00004CC7070050
:1094600010B5040003D10349C420FAF7DDFCA0685D
:1094700010BD000040D4070010B5040003D103491B
:10948000C420FAF7D1FCA06810BD000040D407004A
:1094900010B5040003D10349C420FAF7C5FCA06845
:1094A00010BD000040D4070070B50D46040003D184
:1094B00008495020FAF7B8FC1DB906495120FAF7BF
:1094C000B3FC2560286860602046BDE8704000F06D
:1094D00003B8000050CF070010B5040003D11049B5
:1094E0003320FAF7A1FC206818B90D493420FAF7A7
:1094F0009BFC606818B90A493520FAF795FCD4E955
:1095000000104A68904201D1002004E0D0E9002315
:109510009A4202D01046A06010BD08306060F0E7AB
:1095200050CF070010B5040003D112496320FAF7A9
:109530007BFC206818B90F496420FAF775FCA06815
:10954000002815D0216889680844A060606818B9AF
:1095500008497320FAF768FCD4E901014268914296
:1095600006D1083060602046BDE81040FFF7B4BF68
:1095700010BD000050CF07000C4A10B502F59473DF
:109580000EE0991AC91001EBD171491002EBC1012B
:109590000C68844201D90B4602E005D201F10802B1
:1095A0009A42EED3002010BD486810BD68C4070081
:1095B00000B5FFF7E1FF002800D1014800BD000021
:1095C00054C407002DE9F04104461348134BC01A58
:1095D0000C21B0FBF1F6A0694FF0FF3110F8022C1E
:1095E00002B92169002011E000EB400503EB85057D
:1095F0002F68974209D14F1C02D06F688F4204D167
:1096000094E80F00AD68A84703E0401CB042EBD3DC
:1096100001202060BDE8F0810CD9070000D90700C7
:1096200010B5144612680830202A02D248F21450AD
:1096300010BD002201F030FF0028F9D12020206069
:10964000002010BD083001F0AFBF083002F06EB846
:1096500002480068002800D0012070470004014043
:1096600070B50C46050004D10F494FF48270FAF72B
:10967000DBFB24B90C4940F20510FAF7D5FB0B4887
:109680000B49401AC008042101EB004009A1FFF773
:109690007BFA13490320C96888476869FEF75AFABC
:1096A000FBF7C7FD607070BDDCCA070050D807002B
:1096B00038D8070048616E646C65204E52465F449E
:1096C00046555F4F505F4F424A4543545F435245B2
:1096D0004154452028636F6D6D616E642900000060
:1096E0004C2B002070B50D4620B916494FF49670EA
:1096F000FAF79AFB25B9134940F22D10FAF794FBBB
:1097000011481249401AC108042000EB01400446E8
:109710000FA1FFF739FA1949081FFEF735FAFBF7D1
:1097200088FD6870012805D10020FDF7DDFF10B12C
:109730000A20687070BD2046BDE8704010A1FFF798
:1097400023BA0000DCCA070050D8070038D8070049
:1097500048616E646C65204E52465F4446555F4FCB
:10976000505F4F424A4543545F4558454355544521
:109770002028636F6D6D616E64290000542B0020FA
:1097800057726974696E672076616C696420696ECE
:10979000697420636F6D6D616E6420746F20666CF8
:1097A0006173682E0000000070B50D46040004D1FE
:1097B0001A494FF48970FAF737FB206920B9174925
:1097C00040F21310FAF730FBA08A20B913494FF486
:1097D0008A70FAF729FB25B9104940F21510FAF7FB
:1097E00023FB0F480F49401AC008042101EB004039
:1097F0000DA1FFF7C9F9A18A2069FEF767F9FBF708
:1098000018FD68702846FBF713FAE168002903D0B9
:109810002069BDE87040084770BD0000DCCA070041
:1098200050D8070038D8070048616E646C65204E38
:1098300052465F4446555F4F505F4F424A4543543E
:109840005F57524954452028636F6D6D616E6429DE
:109850000000000030B587B00C46054618221C49B0
:109860006846F8F7DFFD207B01951A4D8DF8000062
:10987000012806D0022817D0062823D1607B049047
:1098800020E0A888E880607B0490217CE08961F377
:109890001F40617C40EA016005900498012811D1C5
:1098A0000D48FDF735FF0DE00C480D49401AC00882
:1098B000042101EB00400BA1FFF766F9B4F80D009D
:1098C000A880E8806846FDF719FC07B030BD0000AD
:1098D000F8C207002C2B002020D8070040D8070032
:1098E00038D8070053657420726563656970742009
:1098F0006E6F74696600000070B50E460B480C4927
:10990000401AC108042000EB01440AA12046FFF7D9
:109910003BF9114D204611A1AB6C2A6DFFF73FF9C1
:10992000A86CB060286D706070BD000050D8070052
:1099300038D8070048616E646C65204E52465F441B
:1099400046555F4F505F4352435F4745542028645C
:109950006174612900000000C04700204F666673F3
:1099600065743A25642C204352433A3078253038C8
:10997000780000002DE9F84F0D4607463748384972
:109980004FF00409401AC40809EB0440064635A10B
:10999000FFF7FAF8FEF76AF9012101EB04444FF0F2
:1099A000080AA8B17A694FF00308B2B137493848BC
:1099B000130515D0436DD1F808C0134463450FD08B
:1099C000204634A1FFF7E0F885F80180BDE8F88F64
:1099D000204639A1FFF7D8F819E0204644A1F1E765
:1099E000B2F5805F06D9204648A1FFF7CDF885F88B
:1099F0000190EBE7436DD1F808C003EB0208E045A6
:109A000008D920464A49CDF800C0FFF7D0F885F8BC
:109A100001A0DBE74264C26C036503638046826495
:109A20007869002200F6FF70070B48683946184431
:109A3000FDF772F930B120463EA1FFF7A5F80520E9
:109A40006870C3E7D8F84810009130463FA1D8F8B5
:109A50005030D8F84420FFF7AAF8B7E750D80700ED
:109A600038D8070048616E646C65204E52465F44EA
:109A700046555F4F505F4F424A4543545F435245FE
:109A80004154452028646174612900004C2B00205A
:109A9000C04700204F626A6563742073697A65204D
:109AA0006D757374206265207061676520616C69F3
:109AB000676E65640000000043616E6E6F74206322
:109AC00072656174652064617461206F626A6563A8
:109AD0007420776974686F75742076616C6964208E
:109AE000696E697420636F6D6D616E6400000000C3
:109AF0004F626A6563742073697A652063616E6E74
:109B00006F7420626520302E00000000496E76617F
:109B10006C69642073697A6520666F72206F626A6F
:109B20006563742028746F6F206C6172676529000B
:109B300068CA07004572617365206F706572617451
:109B4000696F6E206661696C6564000043726561CF
:109B500074696E67206F626A6563742077697468E0
:109B60002073697A653A2025642E204F66667365F6
:109B7000743A203078253038782C204352433A20EC
:109B800030782530387800002DE9F0410E46074640
:109B900015481649401AC508042000EB054014A1D9
:109BA000FEF7F2FF1C4CD4E91401626C431A9A428E
:109BB0000AD0012000EB054018A1FEF7F0FF0820B5
:109BC00070700120BDE8F08100216164A16CE16446
:109BD00060650021384600F035F819490420C9684D
:109BE00088470020EEE7000050D8070038D807006B
:109BF00048616E646C65204E52465F4446555F4F27
:109C0000505F4F424A4543545F455845435554457C
:109C10002028646174612900C0470020496E766184
:109C20006C696420646174612E206578706563746A
:109C300065643A2025642C20676F743A20256400FF
:109C40004C2B0020F0B5044687B00020FEF752FCF4
:109C500001002548254A4FF00107A0EB02004FEA1A
:109C6000D0050AD0224A18212046F9F7C7FF020082
:109C700037D007EB05401FA131E01822284968467C
:109C8000F8F7D0FB2748284E184B174D016DEB1AFB
:109C90000420DB08B26800EB0345914215D1284649
:109CA00022A1FEF771FFD6E90101FDF7EBFD8DF86A
:109CB0000100FBF7BEFA8DF80100D4E901126846F5
:109CC00090472648FDF710FD05E08DF80170D4E9B6
:109CD0000112684690479DF80120284620A1FEF712
:109CE00057FF07B0F0BD000050D8070038D8070074
:109CF000459C07004661696C656420746F2073633E
:109D0000686564756C65206F626A65637420657848
:109D100065637574653A20307825782E0000000060
:109D2000B8C30700C04700204C2B002057686F6C59
:109D300065206669726D7761726520696D6167651E
:109D40002072656365697665642E20506F73747642
:109D5000616C69646174696E672E0000199F070069
:109D6000526571756573742068616E646C696E67A5
:109D700020636F6D706C6574652E20526573756C11
:109D8000743A20307825780038B50D460C480D49D6
:109D9000401AC108042000EB014004460AA1FEF766
:109DA000F3FE134813A1826CAA60036D4FF4805038
:109DB0006B60E86000902046FEF7F9FE38BD0000B9
:109DC00050D8070038D8070048616E646C65204E93
:109DD00052465F4446555F4F505F4F424A45435499
:109DE0005F53454C45435420286461746129000049
:109DF000C0470020637263203D20307825782C20F6
:109E00006F6666736574203D20307825782C206D50
:109E100061785F73697A65203D203078257800008D
:109E20002DE9F0410E46044626482749401AC70846
:109E3000042000EB074025A1FEF7A6FEFDF716FF64
:109E400090B12C4DD5E91401401AA18A6A6C0844DE
:109E500090420BD9012000EB074027A1FEF794FEAA
:109E600003207070BDE8F0810820FAE7284A286BCB
:109E7000526800EB02081F4A20694832FAF7EAFEEE
:109E80000746E06820B923494FF4F870F9F7CCFF92
:109E9000D4E90331A28A4046FCF7F4FF20B1D4E9AB
:109EA0000310BDE8F0410847A18A286B08442863E5
:109EB000A18A286DAF6408442865B760286D70607A
:109EC000D0E7000050D8070038D8070048616E641A
:109ED0006C65204E52465F4446555F4F505F4F427F
:109EE0004A4543545F575249544520286461746180
:109EF00029000000C0470020577269746520726510
:109F0000717565737420746F6F206C6F6E670000DD
:109F10004C2B0020DCCA07000848094910B5401A3C
:109F2000C008042101EB004006A1FEF72DFE1249F6
:109F30000620C968BDE810400847000050D8070057
:109F400038D80700416C6C20666C617368206F70B4
:109F500065726174696F6E73206861766520636FE6
:109F60006D706C657465642E2044465520636F6D7A
:109F7000706C657465642E004C2B0020FEF7BCFEEF
:109F8000FEF792FC0028FBD10D4E64254FF47A4772
:109F9000741C3846A0476D1EFAD10A480068C007F5
:109FA00000D000BEBFF34F8F0648E4380168064A70
:109FB00001F4E06111430160BFF34F8F00BFFDE783
:109FC000A0C00700F0ED00E00400FA0510B504465B
:109FD000084809492246401AC008042101EB004004
:109FE00006A1FEF7D5FD2146BDE810400848FBF765
:109FF00017BE000040D8070038D8070046726565D4
:10A00000696E6720627566666572202570000000C3
:10A01000A8D8070030B58A1D8B79083187B0022B8C
:10A0200033D153888489A3422FD1127A012A2CD1AB
:10A03000184C0DF1040C3CCC8CE83C000A89ADF8BE
:10A040000C204A890C3104911249ADF80E20803958
:10A05000114C096A0591CDF818D0018A05AA6088CB
:10A06000ADDF18B96846FAF72BFC38B10020ADF81F
:10A07000080001A96088B0DF50B106E040F2FD1091
:10A08000ADF8080001A96088B0DF002007B030BD3E
:10A090000120FBE710C307002C2B002070B50646FB
:10A0A0008C1DC888B18888B088422DD11B48FBF729
:10A0B00051FD05001A481B49A0EB01004FEAD000F2
:10A0C00024D0F4210091042101EB004063892A4649
:10A0D00015A1FEF76CFD628904F10C012846F8F722
:10A0E000A1F91822184901A8F8F79CF902960595DC
:10A0F0006089ADF8180001A8FDF700F8002803D02A
:10A1000029460648FBF78CFD08B070BD022101EB23
:10A1100000400EA1FEF738FDF6E70000A8D80700C2
:10A1200040D8070038D8070042756666657220255A
:10A13000702061637175697265642C206C656E2096
:10A14000256420282564290020C3070063616E6E02
:10A150006F7420616C6C6F63617465206D656D6FE9
:10A16000727920627566666572210000F8B50D4649
:10A1700014460646694600F05DFA00280FD0009BA1
:10A18000B3F5803F0AD2981C834207D8A9780222EF
:10A19000B2EB911F02D02989814201D20020F8BD83
:10A1A0002380A11C3046009A00F09AFBF8BD1146AE
:10A1B00000F0D5B8114600F0E7B8F8B50C461546E2
:10A1C0000646694600F036FA00280CD0009A501C6A
:10A1D000904207D3A1780223B3EB911F02D02189CB
:10A1E000814201D20020F8BD2946304600F078FBBC
:10A1F000009A0021A954F8BD2DE9FF410C46CE6814
:10A2000017460546694600F03DFB00280ED0E06881
:10A2100000280BD0A0783A46C0F30110022831463E
:10A22000684606D000F0DEF80199696004B0BDE828
:10A23000F08100F085F8F7E77CB50D4614466946D5
:10A2400000F095F9002820D02889082806D0042895
:10A2500009D002280AD001280CD015E0DDE9000160
:10A26000C4E900010AE00098206006E0009800B20E
:10A27000208002E0009840B22070C117DDE9002381
:10A2800050405940084301D000207CBD01207CBDD6
:10A290007CB50D461446694600F0A7F9002820D089
:10A2A0002889082807D00021042809D002280AD0CC
:10A2B00001280CD014E0DDE90001C4E9000109E047
:10A2C0000098206006E0009880B2208002E00098AC
:10A2D000C0B22070DDE9002350405940084301D04E
:10A2E00000207CBD01207CBD7CB50D46144669462E
:10A2F00000F07BF9002820D02889082808D0009990
:10A30000CA1704280BD002280CD001280DD013E066
:10A31000DDE90012C4E900120846134608E00846C9
:10A32000216004E008B2208001E048B22070C31729
:10A3300048405340184301D000207CBD01207CBD23
:10A3400070B50D46064614461146284600F0B5FA8B
:10A35000224629463046BDE8704000F043B838B583
:10A360000C460422694600F0BBFA00280BD09DF889
:10A370000210BDF8000061F31F409DF8031040EA91
:10A3800001602060012038BD1CB50C4608226946DA
:10A3900000F0A6FA002824D09DF801109DF80020B6
:10A3A0009DF80230080E42EA012242EA034240EAE6
:10A3B00013409DF803309DF8041040EA1320084331
:10A3C0009DF8051042EA036240EA01209DF806105C
:10A3D00040EA01409DF8071040EA0160C4E900200E
:10A3E00001201CBD2DE9F04F05469DB000200F90C7
:10A3F000064610904FF0FF3A01A800F07FF94FF0A9
:10A40000010B0DF13C0983E012AB6A460BA928460B
:10A4100000F0CAF850B101A8009900F080F960B1CD
:10A420000298807810F0300F54D061E09DF8480019
:10A43000002871D11DB0BDE8F08F0098B04243D321
:10A44000029C01AE0298807800F00F00082812D01C
:10A45000304600F07BF90298A042F3D156460098AE
:10A46000B04231D3D5F8088007909DF82C000E90AB
:10A470000598046821E002980688F0E720680768DC
:10A480002FB1214628460E9B079AB84712E0119536
:10A49000216807980E9F8968098881420CD121465E
:10A4A00017A8FBF76FF984F80CB017AA3946119872
:10A4B000FAF769FC0028BDD0A46814B1A968414529
:10A4C000DCD0A968414523D19DF82C10284600F026
:10A4D00043FA1BE0039840280AD200F01F000BFA51
:10A4E00000F20398400959F82030134349F820300E
:10A4F000EC682CB101AB9DF82C2028460099A047B0
:10A5000001AA9DF82C102846FAF73DFC002891D0AE
:10A51000A86800287FF478AFDDE90204857801A8F7
:10A5200000F014F90028F7D115F0300F03D102988C
:10A53000008800B1641CC4B10020494605E000BF9A
:10A5400051F82020521C0ED1401CB0EB541FF7D301
:10A55000600959F8201004F01F00C0F120022AFA07
:10A5600002F0814201D0002064E7012062E71CB5BF
:10A570000C46694600F039F8002814D0DDE90002E5
:10A58000C10709D051084FEA30006FEA00026FEAB4
:10A590000100C4E9002004E051084FEA3000C4E99A
:10A5A00000014FF001001CBDF8B5074600201870EF
:10A5B00008700E4610601C4615466946384600F085
:10A5C00039F801004FF0010009D0009959B1C808CD
:10A5D0002860009800F0070030700120F8BDB968CD
:10A5E00009B10020F8BD2070FBE72DE9F8430026F3
:10A5F000884681463446354604E0402E02D300208A
:10A60000BDE8F8836946484600F096F90028F7D07F
:10A610009DF80070324607F07F00C10FF7F7EEFE9D
:10A6200029430443F61D0D463806E6D4C8E9004127
:10A630000120E5E7F8B50E460746694600F07CF9CB
:10A6400000280AD09DF80040200616D5072504F002
:10A650007F0403E0202D01D30020F8BD6946384671
:10A6600000F06AF90028F8D09DF8001001F07F0092
:10A67000A8400443ED1D0806ECD401203460F8BD69
:10A6800030B45968114AC968914208D1D0E9011221
:10A690000F48D0E90134234303D00021817030BC3E
:10A6A000704711F8013BA2F101021B06F9D4C0E981
:10A6B0000112012181700748074930BC401AC008C7
:10A6C000042101EB004005A1FEF762BA40C107007A
:10A6D000602B002068D8070038D8070050423A2085
:10A6E000496E6974207061636B6574206461746184
:10A6F000206C656E3A20256400000000C2600023D3
:10A700000160C0E901138B881A440261B1F9063077
:10A710001A4442610888002800D00120704770B5B3
:10A7200045680E46044660680188B14206D18078CB
:10A7300000F00F00082801D0012070BD204600F075
:10A7400005F86068A842EED1002070BD30B54168C0
:10A750000A885AB101F1100343600A8A42B18C7829
:10A760000A89C4F30115032D07D00BE0002030BD8A
:10A77000C2680168FFF7C2FFF8E79D78C5F30115CD
:10A78000032D06D00225B5EB141F08D14C89624376
:10A7900009E08D8804690022641B046103E0B5EBC5
:10A7A000941F00D10422897811F0300F02D1816802
:10A7B000491C81609C880169214411440161B3F9FD
:10A7C000062011444161012030BD30B541680024AC
:10A7D00087B0897801F00F02082A11D08A091ED0AB
:10A7E0000222B2EB911F09D10269C1F301110229C2
:10A7F000146001D0032901D14069048007B030BD45
:10A800000069056808E02C7329466846FAF7BAFF24
:10A810006846FFF7DAFFAD68002DF4D1EEE7C1F32B
:10A820000111012912D00229E6D00329E4D042689F
:10A83000917801F00F0107290BD0D16881B11289FD
:10A84000006907B0BDE83040F7F7ECBD41690C7016
:10A85000EDE70169D06807B0BDE8304000F02DB8E1
:10A860001189006907B0BDE83040F7F7F4BD00007A
:10A8700010B5034B002408C080E8160010BD00008E
:10A88000CD4B070038B50D4604466946FFF7D2FEAA
:10A8900000280BD0D4E90002D4E90213C5E9000274
:10A8A000C5E902130098814201D2002038BDA8609A
:10A8B000A168081AA060012038BD00B50A4687B01B
:10A8C00001466846FFF71AFF002807D06846FFF7E1
:10A8D0007CFF6846FFF73AFF0028F7D107B000BDBC
:10A8E0007FB514460546A9B9124A2868904208D196
:10A8F00010E0102269462846FFF7F2FF002807D033
:10A90000103C102CF5D8224669462846FFF7E8FF90
:10A9100004B070BDA868A04201D20020F8E72B68FF
:10A920002246284698470028F2D0A868001BA86055
:10A930000120EDE7CD4B070010B5044680680028E4
:10A9400009D02368012220469847002803D0A06838
:10A95000401EA060012010BD38B5002439B1012986
:10A9600012D0022912D005291DD0002038BD05467D
:10A97000012269462846FFF7B3FF90B19DF8000019
:10A980000006F5D4012038BD08220DE005466946D1
:10A99000FFF750FE28B100212846009AFFF7A0FFDC
:10A9A00038BD204638BD0422BDE838400021FFF7FD
:10A9B00097BF000010B50C46017A052908D0407AEF
:10A9C00038B1084808A102682046FDF76DFB00E099
:10A9D0001AB106A12046FDF767FB2046BDE81040EE
:10A9E000FDF7A0BBC82B0020257300000D0A000056
:10A9F0002DE9FC418046224817460E46C5680A46A6
:10AA0000012441462846FAF735FC70B195F8550007
:10AA100068B100F00101C0F3400243462846CDE989
:10AA2000006700F089F848B109E0172407E03B46C9
:10AA300032464146284600F027F8F4E70524114D38
:10AA40006FB1012C13D005F12400FBF7FFFE00BF0E
:10AA5000FCF74EFDC5F848802046BDE8FC81012C7E
:10AA600002D0FCF745FDF7E701206861F4E700221A
:10AA700031464046FAF7EEF8C5E90960E8E700001C
:10AA8000602B0020C04700202DE9F041044690F8DB
:10AA9000550094B01D461746884620B1174940F22C
:10AAA0002730F9F7C1F90126CDE9007643460022A7
:10AAB000214602A8F9F786FF00281CD0D5B1412213
:10AAC00002A90F48F7F7AEFC0F4810490D4D401A88
:10AAD000C008042101EB00400DA1EE62FEF754F81E
:10AAE0000020286294F8920010B194F8930008B9FD
:10AAF0006068A860012014B0BDE8F081BCCE0700FA
:10AB0000614A0020C047002068D8070038D80700F5
:10AB1000496E76616C69646174696E67206F6C64FC
:10AB2000206170706C69636174696F6E20696E205A
:10AB300062616E6B20302E002DE9FF4FA5B0884674
:10AB400004461546442113A8329FF7F784FC44219C
:10AB500002A8F7F780FCDDF8A09058EA050004D1C0
:10AB60003C4940F26130F9F75FF93B483B4A801AB3
:10AB700002224FEAD00A02EB0A46B8F1000F1ED0BB
:10AB8000A16D289800F01CFE002848D02898FAF7FC
:10AB90008FFD4FF0010B20B130463149FDF7F4FF36
:10ABA000B5B3A16DCDE9001B0022214613A8289B57
:10ABB000F9F708FF002832D0A06D81443F1A8DB10B
:10ABC0000020CDE900704B464246214602A8F9F725
:10ABD000F9FE002823D09DF8080018B1304621491D
:10ABE000FDF7D2FF339898B31F4EB8F1000F1ED077
:10ABF0002898FAF75DFD18B106F11800FBF726FE5C
:10AC0000412213A91948F7F70DFC5DB1AC200AE009
:10AC1000FFE70BEB0A401649FDF7B6FF002029B00D
:10AC2000BDE8F08FA520F062A06D706301E0AA205E
:10AC3000F0626DB10D48412202A98230F7F7F2FBB4
:10AC400094F8920010B194F8930008B96068F0602D
:10AC50000120E4E7BCCE070068D8070038D8070019
:10AC600078CE070074CD0700C0470020204A00209E
:10AC7000C0CC070038B5C3880D46044633B114A0D4
:10AC8000009015A216A12846FDF70EFA217A052993
:10AC90001CD0607A48B1A088FDF7D8FD164951F85C
:10ACA000202016A12846FDF7FFF9A0880021FEF715
:10ACB00015F803461049207A143951F8202001B0C4
:10ACC0002846BDE830400EA1FDF7EEB938BD0000C2
:10ACD0001B5B306D000000001B5B313B33316D00AE
:10ACE00025734C6F67732064726F707065642028E1
:10ACF00025642925730D0A00C82B00202573000048
:10AD00003C25733E2025733A20000000EFF30580B8
:10AD1000C005C00D01D001207047EFF3148040F34F
:10AD20000000401C70470000034802490068FAF721
:10AD3000BDBE0000882B002024C407002DE9F0418F
:10AD4000224C0025224E207A012730B92148311D9E
:10AD50000068FAF7B6FE306038B102202072316820
:10AD6000087928B101281CD114E06560BDE8F081A4
:10AD7000D1E90503C01A142800D31420B7EB900FB3
:10AD800001D2820800E001220869C9681844194408
:10AD900029DF03E0D1E90301084428DF58B1112875
:10ADA00012D003213068FAF71AFA25726560BDE8FF
:10ADB000F041FFF7B9BF207C0028D7D1BDE8F041B2
:10ADC00000210220FDF7DABB2772CFE72C510020CB
:10ADD000842B002024C4070010B5074C201DFAF76F
:10ADE0008FFE002806D1607C002803D1BDE810400A
:10ADF000FFF7A4BF10BD00002C51002010B5104675
:10AE00001A46F7F70FFB002010BD10B510461A4682
:10AE1000F7F708FB002010BD2DE9F0411E681C4625
:10AE20001546074621B1012918D0052923D119E07B
:10AE300000202060401C2060B0421CD8012229461E
:10AE40003846FFF74DFD002806D015F8010B000627
:10AE500001D52068EEE70120BDE8F0810820024618
:10AE6000186002E004200246186029463846BDE812
:10AE7000F041FFF735BD0020EEE770B516460A46F3
:10AE80000446C11C104600F023FF054661193046F8
:10AE9000C91C00F01DFF284470BD000003B5094A1D
:10AEA00085B0D2E91612CDE9001207498989ADF8BB
:10AEB000001006A9CDE90210044869464088AEDFBB
:10AEC00007B000BD90C20700643000202C2B00208A
:10AED00008467047084670472DE9F047FCF714FC18
:10AEE000DFF8C480D8F83020D8F8347000EB020ABC
:10AEF000B81A411EC1F30B01401A00F6FF792B4925
:10AF00002B48D8F84860081AC508042000EB054013
:10AF1000044628A1FDF738FE42F204002F4A815969
:10AF2000012000EB0545914206D028462CA1FDF7F3
:10AF30002BFE0320BDE8F087D8F830000644B84265
:10AF400005D1204633A1FDF71FFE0020F2E7C0B96E
:10AF500006F500500178142901D9416900E000216B
:10AF60003148B1FBF0F34FF440510A78142A01D96B
:10AF7000496900E00021B1FBF0F220462BA1FDF76A
:10AF80000EFE08234A4631465046FAF719FA0400E5
:10AF900005D0284630A1FDF7F7FD2046CAE7BDE8F9
:10AFA000F0470020FCF7A0BBC047002088D807006E
:10AFB00038D80700456E746572206E72665F626FE6
:10AFC0006F746C6F616465725F6466755F73645FF4
:10AFD000636F6E74696E756500000000DBE5B1514A
:10AFE000536F757263652061646472657373206466
:10AFF0006F6573206E6F7420636F6E7461696E206D
:10B00000612076616C696420536F6674446576696B
:10B0100063652E00534420616C726561647920631E
:10B020006F7069656400000040420F0055706461F4
:10B0300074696E672053442E204F6C642053442063
:10B040007665723A2025642C204E657720766572ED
:10B050003A202564000000004661696C6564207434
:10B060006F20636F7079206669726D776172652EEB
:10B070000000000070B50F480F49401AC4080420B2
:10B0800000EB04400DA1FDF77FFDFFF725FF050054
:10B090004FF0010000EB044402D020460FA105E070
:10B0A000F8F7CCFE050004D0204612A1FDF76CFD98
:10B0B000284670BD88D8070038D80700456E7465EB
:10B0C00072206E72665F6466755F73645F626C5F48
:10B0D000636F6E74696E75650000000053442B4207
:10B0E0004C3A20534420636F7079206661696C6527
:10B0F0006400000053442B424C3A20424C20636FC2
:10B100007079206661696C6564000000F0B50546E1
:10B11000002003464FF440540C4E4FF6FE7712E0E9
:10B12000D4F804C0B44505D155F823C0B4F80CE0F8
:10B13000F44504D02AB155F823C0BC4501D1012003
:10B14000F0BD5B1CDBB28B42EAD3F0BDDBE5B15155
:10B1500010B5040003D11A495320F8F765FE4FF4E7
:10B16000405018494068884221D1218A71B16269F2
:10B1700004F11400002A94F855200BD0042A07D0BB
:10B180000022BDE81040C9B2FFF7C0BF002010BDCB
:10B190000122F6E712B1012A07D1F7E7012904D904
:10B1A000C9B20022FFF7B2FFF0E7012010BD208AEC
:10B1B00010B160690028E9D120780028F5D110BDD0
:10B1C00004CF0700DBE5B1513EB504460B496846A4
:10B1D000FEF76AF90AE06846FEF742F9D0E9002175
:10B1E0002046904740B16846FEF79CF96846FEF756
:10B1F00037F90028EFD13EBD11203EBDC8C607007B
:10B200003EB504460A496846FEF74EF909E068462D
:10B21000FEF726F9D0E90021204690476846FEF760
:10B2200081F96846FEF71CF90028F0D13EBD000008
:10B23000D4C607002DE9F0411400884618D0002537
:10B240000E4F032608EB050122460020F8F75AF9B5
:10B250000544241A40B93878002809D008494FF429
:10B260007A408847761E05D001203870002CE9D13D
:10B27000BDE8F08100203870FAE700008C2B002038
:10B28000A1C607002DE9F0410E46074613481449B0
:10B29000144D401AC408032000EB044012A12A6890
:10B2A000FDF776FC3046F9F7F3FC20B919494FF465
:10B2B000C170F8F7B9FD184B3A463146286800F0DE
:10B2C00053F8020007D0012000EB0440BDE8F04134
:10B2D00012A1FDF75DBCBDE8F081000058D8070061
:10B2E00038D807005C2B00204261636B696E6720D1
:10B2F00075702073657474696E677320706167651B
:10B3000020746F20616464726573732030782578CF
:10B310002E00000034CC070040440020436F756CC1
:10B3200064206E6F7420706572666F726D2062614A
:10B33000636B7570206F6620626F6F746C6F6164F1
:10B3400065722073657474696E677321204572722B
:10B350006F723A20307825780000000000225821D2
:10B36000001DF9F777BC00002DE9F04715464FF4B2
:10B3700060771E46894680463A46F7F77EF8224AAD
:10B38000224B0421D21AD20801EB024400282046A5
:10B3900017D01FA1FDF7F8FB2046424621A1FDF77B
:10B3A000F7FB002201214046FBF7B6FC174A164B7B
:10B3B00001219A1AD20801EB024458B1204621A17A
:10B3C0001DE02949FDF7E0FB0DB10020A847002052
:10B3D000BDE8F08726B9254940F25D10F8F724FD55
:10B3E0003A4649463046F7F71DF82B463A4631466D
:10B3F0004046FBF747FD0028EAD020461CA1FDF798
:10B40000C3FB0320E4E7000058D8070038D8070042
:10B4100057726974696E672073657474696E6773B7
:10B420002E2E2E0045726173696E67206F6C64204A
:10B4300073657474696E67732061743A203078257F
:10B4400030387800436F756C64206E6F74206572BD
:10B45000617365207468652073657474696E6773C1
:10B460002070616765210000E8CB070034CC07003D
:10B47000436F756C64206E6F7420777269746520F9
:10B48000746865204446552073657474696E6773EB
:10B49000207061676521000070B516460D460400F6
:10B4A00007D035B1206C802200213828225403D3E4
:10B4B00007E00E2070BD2154401C3828FBD30BE060
:10B4C0002154401C4028FBD32146084600F096F842
:10B4D00038212046F6F7BFFF216CD4E912304A0F1D
:10B4E000C900383459185041C4E90410227CE27173
:10B4F0000A0A42EA0062A2710A0C42EA0042627140
:10B50000020242EA116020716069E070010AA170D4
:10B51000010C6170000E04F838092146084600F05D
:10B520006DF84FF00002EEB1E06ED100C840A854B3
:10B53000A36ECB40A8180371636ECB400372236ED9
:10B54000CB400373E36DCB400374A36DCB40037515
:10B55000636DCB400376236DCB40521C0377042AE6
:10B56000E2D31FE018235042216D03EBC000C1401D
:10B57000A954666DC640A9180E71A66DC6400E721C
:10B58000E66DC6400E73266EC6400E74666EC640EB
:10B590000E75A66EC6400E76E66EC640521C0E773D
:10B5A000042AE0D3002070BDA8B100210164C0E9E5
:10B5B00012110A4901650A4941650A4981650A492A
:10B5C000C1650A4901660A4941660A4981660A4914
:10B5D000C166002070470E207047000067E6096AC8
:10B5E00085AE67BB72F36E3C3AF54FA57F520E51A4
:10B5F0008C68059BABD9831F19CDE05B2DE9F04F1B
:10B60000C8B0002213466F46CC181B1D2588A678AB
:10B610006DBA2D04E47845EA0625254347F8225003
:10B62000521C102AF0D31BE007EB820151F8083CB2
:10B630004FEA734484EAF34484EA932451F83C3C8F
:10B640004FEAF31585EAB34585EAD303234451F85D
:10B650001C4C51F8401C2144194447F82210521C3C
:10B66000402AE1D3036D4793416D4691846D459423
:10B67000C26D44929246026E4392456E4295A9462F
:10B68000856E4195C66E4096B34600264FEAB217C6
:10B6900087EAF22787EA726C02EA090725EA0208BC
:10B6A00087EA0807BC44204F57F8268008EB0B07B1
:10B6B000BC445DF82670AB460CEB070E4FEAB307AF
:10B6C00087EA733787EAB35C81EA04074D4601EAEB
:10B6D000040891461F400AEB0E02A24687EA0807BB
:10B6E0000C46BC441946761C0EEB0C03402ECDD301
:10B6F000479E33440365469B19444165459921445F
:10B70000816544995144C165439911440166429948
:10B710004944416641992944816640995944C1662A
:10B7200048B0BDE8F08F000090C507002DE9F0415A
:10B7300016460F46040004D006B317B10025A846EC
:10B740001AE00E20BDE8F081216C785D6054206C19
:10B75000401C206440280ED121460846FFF74EFFCA
:10B76000D4E912014FF40072801841F10001C4F8CD
:10B770004080C4E912016D1CB542E5D30020E1E729
:10B7800010B51620F8F736F848B10C4882684FF427
:10B79000800152B1016821F48001016010BDBDE853
:10B7A000104042F20100F8F76DB94FF0E020C0F808
:10B7B0008011BFF34F8FBFF36F8F10BD344F002048
:10B7C0002DE9F04100F500521A481B4F0123C01B20
:10B7D000174CC008556803EB0040A54201D017493B
:10B7E0001FE04D1EC5F30B05491B41F6FF7596681A
:10B7F00029448E4201D2124913E04FF440514D6862
:10B80000A54211D10C78102C01D9096900E0002162
:10B810001478102C01D9126900E00022914203D063
:10B820000849FDF7B1F900231846BDE8F081000092
:10B83000DBE5B15168D8070038D8070024CE0700EF
:10B84000B8CD070004CD070010B51620F7F7D2FFDA
:10B85000A0B1114890F800044009082811D2012134
:10B86000814011F0EC0F0CD00C4882684FF480013D
:10B870006AB1016841F48001016010BD42F201002B
:10B8800001E042F20200BDE81040F8F7FBB84FF0CB
:10B89000E020C0F8001110BD16E000E0344F002099
:10B8A0002DE9F0471E46924689460546040C089F3E
:10B8B000F9F726FC8046FDF707FAA04204D80FA14D
:10B8C00040F2A910F8F7B0FA44EA0841741C1B488A
:10B8D0003C4000EB84023E4000EB8600D160C16832
:10B8E00065F3C5016AF3891169F39F2121F0030112
:10B8F000491C21F00401C160BDE8F0872E2E5C2EAA
:10B900002E5C2E2E5C2E2E5C2E2E5C636F6D706F67
:10B910006E656E74735C6C69627261726965735C8A
:10B920006C6F675C7372635C6E72665F6C6F675F8F
:10B9300066726F6E74656E642E630000D8520020CC
:10B940002DE9FC47814617481746884605681C467E
:10B95000012201A91846F9F7EDF8134EB8B1019983
:10B960008B1C00200AE000BF57F8202003EA050CDA
:10B9700006EB8C0C401C5B1CCCF80C20A042F3D3D3
:10B980000B462246414648460095FFF789FF30782E
:10B9900002E000BFFCF788FF0028FBD1F9F709FFA0
:10B9A000BDE8FC87982B0020D85200202DE9FF41EC
:10B9B000324800F15C01826B6846FEF759FF304F58
:10B9C0009DE8070007F11C032F4C83E80700194688
:10B9D0002C48C8600020A0706060A0604FF44771E0
:10B9E000A7F54070F6F737FDA7F54072274902F535
:10B9F0004770FEF7A5FC2649264A891AC908012284
:10BA000002EB014578B1A07838B1A7F5407090F805
:10BA10006C110029017826D041B128461EA100BF33
:10BA2000FDF7B2F828E0284623A1F9E790F8720163
:10BA300010B3D4E901122C4E6846FEF719FF9DE8B9
:10BA40000F001C3787E80F004FF4B2713046F6F74D
:10BA500002FD3246254906F5D470FEF771FC30B977
:10BA6000284623A1DCE739B1807928B12F4E012087
:10BA7000E66004B0BDE8F0810020FAE7C04700208E
:10BA8000404E002081A60700602B002060C2070006
:10BA900068D8070038D8070048616E646C65723A50
:10BAA00020496E76616C696420696E697420636FE9
:10BAB0006D6D616E642E000048616E646C65723A53
:10BAC00020496E76616C69642070726F746F636F69
:10BAD0006C20627566666572206D5F70625F73745C
:10BAE0007265616D00000000B44C002040C1070089
:10BAF00048616E646C65723A20496E76616C696467
:10BB00002070726F746F636F6C2062756666657209
:10BB1000206D5F70625F73747265616D2028696E5D
:10BB2000697420636F6D6D616E642900484B00205D
:10BB30002DE9F0410F460546234824492A46401A7C
:10BB4000C008042101EB004021A1FDF721F8B7F165
:10BB5000807F03D324498F20F8F766F9962F03D20C
:10BB600021499020F8F760F96FF07F40874200D2BA
:10BB700038461E4ED6F804150144381A21F07F4489
:10BB8000411E6860952902D29630963C68602D7BF4
:10BB9000042D03D314497720F8F746F906EB850006
:10BBA000C0F8404512494FF4F86088474FF4A07040
:10BBB00000EB85013046FDF729FA4FF48030A840AC
:10BBC000C6F80403BDE8F08188D8070038D807001C
:10BBD00074696D65725F616374697661746520284C
:10BBE000307825782900000054C807000040024042
:10BBF000B1C0070070B5174E3078002829D116481B
:10BC000000680125C0F3004008B914480560144CD1
:10BC10004FF480712046FDF7F9F94FF4A0712046EA
:10BC2000FDF7F4F94FF4A2712046FDF7EFF90D4A44
:10BC30000020A02182F800140A4A1021203AC2F8FC
:10BC40000011C4F80805A56025600220C4F80403AB
:10BC5000357070BDF42A0020180400400800004030
:10BC60000040024024E000E070B515460E46044650
:10BC7000FFF7C0FF314620462560BDE87040FFF762
:10BC800057BF000010B5044609480A492246401A29
:10BC9000C008042101EB004007A1FCF779FF217BDC
:10BCA0004FF4803088400949C1F8080310BD0000F6
:10BCB00088D8070038D8070074696D65725F73749F
:10BCC0006F7020283078257829000000004002405D
:10BCD0000870020A4A70020C8A70000EC8700420B4
:10BCE0007047000010B50248F9F701FF002010BDB1
:10BCF000802B002010B514210448F6F7ACFB044853
:10BD00000068F9F7ADFE002010BD00002C510020A6
:10BD100024C407002DE9F05F8346DDE90A4A99460D
:10BD200090460D460846012703E000BFB0FBF8F03F
:10BD30007F1C4045FAD2B94500D94F465FEACA7028
:10BD400012D18CB15FEA8A7002D5B9F1000F01D02F
:10BD5000202607E0302605E031465846641EF8F7F5
:10BD600043FF0CB1A742F7D35FF00106B9F1010F11
:10BD700002D9A9F1010903E0B5FBF6F0404502D371
:10BD800006FB08F6F2E7DFF83C9000BFB5FBF6F0E3
:10BD900000FB165519F800105846F8F725FFB6FBBA
:10BDA000F8F6002EF2D15FEACA7009D0002C07D055
:10BDB000A74205D220215846641EF8F715FFF5E783
:10BDC000BDE8F09FE8C307002DE9F04108460124D3
:10BDD0001646254600212B460A46FAF741FD0C4936
:10BDE0000C4A891ACF0830B105EB07400AA1FCF7CD
:10BDF000CBFE042409E0FAF719FD02463060042066
:10BE000000EB07400BA1FCF7C3FE2046BDE8F08124
:10BE100068D8070038D8070043616E277420666928
:10BE20006E6420726F6F6D20666F72207570646132
:10BE3000746500005772697465206164647265738B
:10BE4000732073657420746F203078253038780043
:10BE50002DE9F0411C4B1D4F0F2600240125DB1B53
:10BE600090F85520DB0805EB03450AB1042A03D1FD
:10BE700090F86430012B06D0D30707D090F85630E5
:10BE8000012B02D002E0846E0DE0846D92070AD58A
:10BE900090F85C20012A06D1026E0D48C0F5FC2303
:10BEA0009A4204D814443CB101260C6008E02846AC
:10BEB00008A1FCF774FE042628460EA1FCF764FED8
:10BEC0003046BDE8F081000068D8070038D8070088
:10BED00000200700424C2073697A652028256429D8
:10BEE000206F766572206C696D697420282564293D
:10BEF00000000000496E6974207061636B657420F6
:10BF0000646F6573206E6F7420636F6E7461696E09
:10BF10002076616C6964206669726D776172652054
:10BF200073697A650000000030B1006805498842F5
:10BF300005D048F20250704748F201507047002087
:10BF4000704700006E52464870B5FDF781FB00282F
:10BF500011D00020084A094B094C0121166801FA4A
:10BF600000F52E4203D004EB8005C5F80036401CD6
:10BF7000C0B20728F2D370BD080501403546526EA5
:10BF8000000001400748084910B5401AC0080321C5
:10BF900001EB004005A1FCF7F7FDBDE81040FFF7FD
:10BFA000D3BF000038D8070038D80700496E746541
:10BFB000726E616C20666565640000000020704749
:10BFC000002070472DE9FC4180461C4617460E466E
:10BFD0000C48089DF9F794FD10B11120BDE8FC81D3
:10BFE000A20839463046FCF7E1FF0648F9F77FFD25
:10BFF00033463A4601214046CDE90045F9F7D4F8E9
:10C000000020EBE7802B00202DE9F84F114D8846EA
:10C0100081461E4617466946DDF828A02868F9F7CC
:10C020003AFD040013D01C21F6F715FA0020207108
:10C03000C4F80090C4E90486C4E902A769462868E8
:10C04000F9F74AFDFEF7C8FE0020BDE8F88F04208E
:10C05000FBE7000024C407005DE7294771AD136AC0
:10C0600095ACA322B285708EB41556EBAE7D24FF3D
:10C07000BF027B23FD12AB6504AC9F35BED6259273
:10C08000C9063C039151550A5FD2F14C94D11D2150
:10C09000DBAAF5635444CE7A0000000000000000E3
:10C0A0000338FDD8704700000000000000000000C9
:10C0B0000338FDD870470000459607004B960700EF
:10C0C000219607002000000078000000000000001A
:10C0D0004800280000204000C127070000000000A1
:10C0E000010001000000000001000000000000004D
:10C0F0000200050001000000220000000000000016
:10C10000000000000000000000000000000000002F
:10C11000010001000000000001000000000000001C
:10C1200002000500010000004200000000000000C5
:10C1300000000000000000000000000000000000FF
:10C14000010011000400FCFF0400000000000000DA
:10C15000020011000400FCFF0400000000000000C9
:10C16000030021000400FCFF040010000000000098
:10C17000040011000100FFFF0100000000000000AA
:10C18000050011000200FEFF040000000000000096
:10C19000060011000400FCFF040000000000000085
:10C1A000070011000400FCFF040000000000000074
:10C1B000080017000200FEFF24000000E0C0070096
:10C1C000090010000100FFFF01000000DCC00700B3
:10C1D0000A0027000200FEFF4400030010C1070010
:10C1E000000000000000000000000000000000004F
:10C1F000010011000100FFFF01000000000000002D
:10C20000020017000200FEFF6401000040C10700A9
:10C21000000000000000000000000000000000001E
:10C22000010007000000000068010000F0C10700E5
:10C2300002000100000000000100000000000000FA
:10C2400003000500010000004200000000000000A3
:10C2500000000000000000000000000000000000DE
:10C26000010017000400FCFF68010000F0C1070096
:10C27000020017000400FCFFAC01000020C2070010
:10C2800000000000000000000000000000000000AE
:10C290000011030000111300020000000100000063
:10C2A0000338FDD870470C000C0000005802000055
:10C2B000020000000000000002000000000000007A
:10C2C00028300020090000000000000000000000ED
:10C2D0000100000000000000280000000000000035
:10C2E000000000000001000000000100000000004C
:10C2F000000000000000000000000000000000003E
:10C300006540070000000000000000000000000081
:10C31000020000000000010000000000000000001A
:10C32000080000000000000065400700CD9F0700E6
:10C3300000000000000000000400000000000000F9
:10C3400000000000000000000000000000000000ED
:10C3500000000000000000000000000000000000DD
:10C36000F4000000000000001800000000000000C1
:10C3700000000000000000000000000000000000BD
:10C3800000000000000000000000000000000000AD
:10C39000170000000000000050EADA308883B89FE0
:10C3A000604F15F30000C98E02000000000000007D
:10C3B0000000000000000000040000000000000079
:10C3C000000000000000000000000000000000006D
:10C3D000000100000000000000000000000000005C
:10C3E00000000000000000003031323334353637B1
:10C3F0003839414243444546001000000400000023
:10C400000100000071550700E5BC0700FDAD070005
:10C41000C5BF070015510700D1AE0700BDBF07001B
:10C4200091560700404F002000100000040000005B
:10C43000010000007D550700F5BC07000BAE0700AA
:10C4400009C007005D510700D5AE0700C1BF070056
:10C45000A1560700556E6B6E6F776E206572726F16
:10C460007220636F64650000000000001CD30700A9
:10C4700001000000C8D1070002000000BCCF070087
:10C48000030000003CD207000400000090D2070027
:10C490000500000070D10700060000000CD1070065
:10C4A0000700000078D207000800000084D10700D0
:10C4B00009000000E8D107000A00000004D30700CB
:10C4C0000B000000A4CF07000C0000009CD1070067
:10C4D0000D0000006CD307000E00000068D20700BA
:10C4E0000F000000A4D2070010000000D8D20700FF
:10C4F0001100000080D307001200000054D3070091
:10C5000013000000F0D207008000000024D10700D3
:10C510008100000060D007008200000020D00700EA
:10C520008300000000D00700840000003CD007001A
:10C530008500000048D107008600000050D20700A7
:10C5400090000000ECD0070091000000E0CF070051
:10C5500092000000B0D1070000820000B8D20700AE
:10C560000182000004D207000282000020D20700EE
:10C57000008400007CD007000184000028D307005D
:10C5800002840000C4D0070003840000A0D007008C
:10C59000982F8A4291443771CFFBC0B5A5DBB5E92E
:10C5A0005BC25639F111F159A4823F92D55E1CABA2
:10C5B00098AA07D8015B8312BE853124C37D0C5530
:10C5C000745DBE72FEB1DE80A706DC9B74F19BC178
:10C5D000C1699BE48647BEEFC69DC10FCCA10C2468
:10C5E0006F2CE92DAA84744ADCA9B05CDA88F9764C
:10C5F00052513E986DC631A8C82703B0C77F59BFB6
:10C60000F30BE0C64791A7D55163CA0667292914E1
:10C61000850AB72738211B2EFC6D2C4D130D38537E
:10C6200054730A65BB0A6A762EC9C281852C729240
:10C63000A1E8BFA24B661AA8708B4BC2A3516CC76E
:10C6400019E892D1240699D685350EF470A06A10A7
:10C6500016C1A419086C371E4C774827B5BCB034F6
:10C66000B30C1C394AAAD84E4FCA9C5BF36F2E6894
:10C67000EE828F746F63A5781478C8840802C78C23
:10C68000FAFFBE90EB6C50A4F7A3F9BEF27871C626
:10C69000718707006F8707006987070000000000A7
:10C6A0000338FDD870470000405200207F00000092
:10C6B000C0520020D8D80700E0D8070000000000D2
:10C6C0000000000000100201B4C60700C4C6070045
:10C6D00008000000ECC60700FCC6070008000000C8
:10C6E000FCC607000CC7070008000000F8D80700C8
:10C6F00000D907000000000000000000E8D8070093
:10C70000F8D8070000000000000000000000000052
:10C71000000000000000000000000000D0D807006A
:10C72000D8D807000000000000000000E82A002020
:10C730000CC707002CC7070008000000E0D807005E
:10C74000E8D8070000000000000000003CC7070018
:10C750004CC7070008000000E9A2070091A20700EB
:10C7600039A20700AFA10700B5A107006DA107001E
:10C77000BBA10700F9A107000000000000404040F5
:10C7800040404040404041414141414040404040A4
:10C790004040404040404040404040404005020250
:10C7A000020202020202020202020202022020200F
:10C7B000202020202020200202020202020290906B
:10C7C0009090909010101010101010101010101069
:10C7D00010101010101010100202020202028888BD
:10C7E00088888888080808080808080808080808C9
:10C7F00008080808080808080202020240000000B1
:10C800007DC707002E2E5C2E2E5C2E2E5C2E2E5CFD
:10C810002E2E5C636F6D706F6E656E74735C6C69E9
:10C82000627261726965735C626F6F746C6F616470
:10C8300065725C6E72665F626F6F746C6F61646567
:10C84000725F6170705F73746172745F66696E614C
:10C850006C2E63002E2E5C2E2E5C2E2E5C2E2E5CFB
:10C860002E2E5C636F6D706F6E656E74735C6C6999
:10C87000627261726965735C626F6F746C6F616420
:10C8800065725C6E72665F626F6F746C6F61646517
:10C89000725F6466755F74696D6572732E63000004
:10C8A0002E2E5C2E2E5C2E2E5C2E2E5C2E2E5C638D
:10C8B0006F6D706F6E656E74735C6C6962726172BD
:10C8C0006965735C626F6F746C6F616465725C6ED6
:10C8D00072665F626F6F746C6F616465725F6677BA
:10C8E0005F61637469766174696F6E2E6300000026
:10C8F00043524320636F6D7075746174696F6E206D
:10C900006661696C656420666F7220636F7069652B
:10C9100064206170703A20737263206372633A20FE
:10C920003078253038782C20726573206372633A32
:10C9300020307825303878004120536F6674446584
:10C940007669636520686173206A75737420626517
:10C95000656E206163746976617465642E20497424
:10C960002773206C696B656C792074686174206131
:10C970006E206170706C69636174696F6E20776995
:10C980006C6C20636F6D6520696D6D6564696174A1
:10C99000656C7900526563656976656420424C4533
:10C9A0005F47415454535F4556545F45584348418F
:10C9B0004E47455F4D54555F5245515545535420A0
:10C9C00028726571756573743A2025642C20726530
:10C9D000706C793A202564292E0000002E2E5C2EE2
:10C9E0002E5C2E2E5C2E2E5C2E2E5C636F6D706F77
:10C9F0006E656E74735C6C69627261726965735C9A
:10CA0000626F6F746C6F616465725C626C655F64A9
:10CA100066755C6E72665F6466755F626C652E63D8
:10CA2000000000006E72665F6673746F7261676506
:10CA30005F777269746528616464723D25702C208B
:10CA40007372633D25702C206C656E3D25642062F9
:10CA500079746573292C207175657565207573610E
:10CA600067653A20256400004372656174696E67EA
:10CA700020746865206F626A6563742077697468E2
:10CA80002073697A652030782530387820776F7583
:10CA90006C64206F766572666C6F77206669726D64
:10CAA000776172652073697A652E204F66667365BB
:10CAB000742069732030782530387820616E6420C6
:10CAC0006669726D776172652073697A6520697332
:10CAD000203078253038782E000000002E2E5C2E75
:10CAE0002E5C2E2E5C2E2E5C2E2E5C636F6D706F76
:10CAF0006E656E74735C6C69627261726965735C99
:10CB0000626F6F746C6F616465725C6466755C6E95
:10CB100072665F6466755F7265715F68616E646C92
:10CB200065722E6300000000526573657474696E4F
:10CB30006720626F6F746C6F6164657220736574D7
:10CB400074696E67732073696E6365206E656974BE
:10CB5000686572207468652073657474696E6773A4
:10CB60002070616765206E6F722074686520626155
:10CB7000636B7570206172652076616C6964202832
:10CB8000435243206572726F72292E00526573748E
:10CB90006F72696E672073657474696E677320665F
:10CBA000726F6D206261636B75702073696E63656F
:10CBB000207468652073657474696E677320706192
:10CBC000676520636F6E74656E7473206172652093
:10CBD000696E76616C6964202843524320657272E5
:10CBE0006F72292E0000000044657374696E6174D1
:10CBF000696F6E2073657474696E67732061726506
:10CC0000206964656E746963616C20746F20736F52
:10CC1000757263652C207772697465206E6F74205D
:10CC20006E65656465642E20536B697070696E670C
:10CC30002E0000002E2E5C2E2E5C2E2E5C2E2E5CE6
:10CC40002E2E5C636F6D706F6E656E74735C6C69B5
:10CC5000627261726965735C626F6F746C6F61643C
:10CC600065725C6466755C6E72665F6466755F7340
:10CC7000657474696E67732E630000002E2E5C2E3F
:10CC80002E5C2E2E5C2E2E5C2E2E5C636F6D706FD4
:10CC90006E656E74735C6C69627261726965735CF7
:10CCA000626F6F746C6F616465725C6466755C6EF4
:10CCB00072665F6466755F7574696C732E630000DD
:10CCC0004D616A6F722053442075706461746520F1
:10CCD000627574206E6F20424C2E2041626F727418
:10CCE00020746F2061766F696420696E6361706182
:10CCF0006369746174696E672074686520424C2EA4
:10CD000000000000546865206E657720536F6674DC
:10CD1000446576696365206973206F6620612064CD
:10CD20006966666572656E742066616D696C7920EE
:10CD30007468616E207468652070726573656E74C6
:10CD400020536F66744465766963652E20436F6D6A
:10CD50007061746962696C6974792063616E6E6F69
:10CD6000742062652067756172616E746565642EFA
:10CD700000000000426F6F742076616C696461741A
:10CD8000696F6E206F6620626F6F746C6F6164658F
:10CD900072206973206E6F7420737570706F727477
:10CDA000656420616E642077696C6C20626520691F
:10CDB000676E6F7265642E0054686520536F6674E9
:10CDC0004465766963652073697A6520696E2074AD
:10CDD000686520696E666F2073747275637420696C
:10CDE0007320746F6F20736D616C6C20636F6D7056
:10CDF000617265642077697468207468652073695E
:10CE00007A65207265706F7274656420696E207433
:10CE1000686520696E697420636F6D6D616E642E44
:10CE20000000000054686520536F6674446576699D
:10CE3000636520646F6573206E6F7420636F6E741A
:10CE400061696E20746865206D61676963206E7525
:10CE50006D626572206964656E74696679696E6772
:10CE6000206974206173206120536F667444657675
:10CE70006963652E00000000496E76616C6964612B
:10CE800074696E6720617070206265636175736597
:10CE900020697420697320696E636F6D70617469B5
:10CEA000626C6520776974682074686520536F66CA
:10CEB000744465766963652E000000002E2E5C2E9A
:10CEC0002E5C2E2E5C2E2E5C2E2E5C636F6D706F92
:10CED0006E656E74735C6C69627261726965735CB5
:10CEE000626F6F746C6F616465725C6466755C6EB2
:10CEF00072665F6466755F76616C69646174696FA0
:10CF00006E2E63002E2E5C2E2E5C2E2E5C2E2E5C42
:10CF10002E2E5C636F6D706F6E656E74735C6C69E2
:10CF2000627261726965735C626F6F746C6F616469
:10CF300065725C6466755C6E72665F6466755F766A
:10CF400065725F76616C69646174696F6E2E6300EF
:10CF50002E2E5C2E2E5C2E2E5C2E2E5C2E2E5C63D6
:10CF60006F6D706F6E656E74735C6C696272617206
:10CF70006965735C6578706572696D656E74616C06
:10CF80005F73656374696F6E5F766172735C6E72F6
:10CF9000665F73656374696F6E5F697465722E6333
:10CFA000000000004E52465F4552524F525F494EBC
:10CFB00056414C49445F4441544100004E52465F43
:10CFC0004552524F525F534F46544445564943458C
:10CFD0005F4E4F545F454E41424C454400000000B7
:10CFE0004E52465F4552524F525F4645415455524C
:10CFF000455F4E4F545F454E41424C454400000052
:10D000004E52465F4552524F525F4D555445585F00
:10D01000554E4C4F434B5F4641494C454400000040
:10D020004E52465F4552524F525F4D555445585FE0
:10D030004C4F434B5F4641494C4544004E52465F7E
:10D040004552524F525F4D555445585F434F4E44E1
:10D050005F494E49545F4641494C45440000000039
:10D060004E52465F4552524F525F4D555445585FA0
:10D07000494E49545F4641494C4544004E52465F33
:10D080004552524F525F424C455F495053505F5298
:10D09000585F504B545F5452554E434154454400E1
:10D0A0004E52465F4552524F525F424C455F495087
:10D0B00053505F504545525F52454A45435445449D
:10D0C000000000004E52465F4552524F525F424CA4
:10D0D000455F495053505F4C494E4B5F4449534361
:10D0E0004F4E4E4543544544000000004E52465FAB
:10D0F0004552524F525F4150495F4E4F545F494D28
:10D10000504C454D454E5445440000004E52465F3C
:10D110004552524F525F4E4F545F535550504F52ED
:10D12000544544004E52465F4552524F525F4D4F58
:10D1300044554C455F4E4F545F494E495449414C0C
:10D14000495A4544000000004E52465F4552524F36
:10D15000525F4D4F44554C455F414C5245414459F7
:10D160005F494E495449414C495A4544000000002A
:10D170004E52465F4552524F525F4E4F545F464F9C
:10D18000554E44004E52465F4552524F525F494EF3
:10D1900056414C49445F5354415445004E52465FFA
:10D1A0004552524F525F444154415F53495A4500E2
:10D1B0004E52465F4552524F525F494F5F50454E67
:10D1C00044494E47000000004E52465F4552524FC0
:10D1D000525F5356435F48414E444C45525F4D4960
:10D1E0005353494E470000004E52465F4552524F3E
:10D1F000525F494E56414C49445F4C454E47544856
:10D20000000000004E52465F4552524F525F44525A
:10D21000565F5457495F4552525F414E41434B0060
:10D220004E52465F4552524F525F4452565F5457DA
:10D23000495F4552525F444E41434B004E52465F58
:10D240004552524F525F494E5445524E414C000098
:10D250004E52465F4552524F525F53544F524147D0
:10D26000455F46554C4C00004E52465F4552524F6A
:10D27000525F4E554C4C00004E52465F4552524F45
:10D28000525F494E56414C49445F504152414D0016
:10D290004E52465F4552524F525F4E4F5F4D454D85
:10D2A000000000004E52465F4552524F525F464FBB
:10D2B0005242494444454E004E52465F4552524FF9
:10D2C000525F4452565F5457495F4552525F4F5622
:10D2D000455252554E0000004E52465F4552524F45
:10D2E000525F494E56414C49445F4144445200000C
:10D2F0004E52465F4552524F525F5245534F555220
:10D30000434553004E52465F4552524F525F494E7D
:10D3100056414C49445F464C414753004E52465F8C
:10D3200053554343455353004E52465F4552524F67
:10D33000525F424C455F495053505F4348414E4E07
:10D34000454C5F414C52454144595F4558495354FF
:10D35000530000004E52465F4552524F525F434FBA
:10D360004E4E5F434F554E54000000004E52465FF4
:10D370004552524F525F54494D454F55540000009D
:10D380004E52465F4552524F525F4255535900002C
:10D390002E2E5C2E2E5C2E2E5C2E2E5C2E2E5C6392
:10D3A0006F6D706F6E656E74735C6C6962726172C2
:10D3B0006965735C6C6F675C7372635C6E72665FE9
:10D3C0006C6F675F64656661756C745F6261636BE7
:10D3D000656E64732E6300007761726E696E67001C
:10D3E00064656275670000001B5B313B33306D0084
:10D3F0001B5B306D000000001B5B313B33316D0067
:10D400001B5B313B33326D001B5B313B33336D00B3
:10D410001B5B313B33346D001B5B313B33356D009F
:10D420001B5B313B33366D001B5B313B33376D008B
:10D43000696E666F000000006572726F7200000016
:10D440002E2E5C2E2E5C2E2E5C2E2E5C2E2E5C63E1
:10D450006F6D706F6E656E74735C6C696272617211
:10D460006965735C6578706572696D656E74616C11
:10D470005F73656374696F6E5F766172735C6E7201
:10D48000665F73656374696F6E5F697465722E6839
:10D490000000000073645F626C655F6366675F73C2
:10D4A000657428292072657475726E656420257311
:10D4B000207768656E20617474656D7074696E673D
:10D4C00020746F2073657420424C455F474154546B
:10D4D000535F4346475F534552564943455F434870
:10D4E000414E4745442E000073645F626C655F6384
:10D4F00066675F73657428292072657475726E653E
:10D5000064202573207768656E20617474656D7082
:10D5100074696E6720746F2073657420424C455F98
:10D52000434F4D4D4F4E5F4346475F56535F5555F2
:10D5300049442E0073645F626C655F6366675F7366
:10D54000657428292072657475726E656420257370
:10D55000207768656E20617474656D7074696E679C
:10D5600020746F2073657420424C455F47415454CA
:10D57000535F4346475F415454525F5441425F53A7
:10D58000495A452E0000000073645F626C655F635A
:10D5900066675F73657428292072657475726E659D
:10D5A00064202573207768656E20617474656D70E2
:10D5B00074696E6720746F2073657420424C455FF8
:10D5C000434F4E4E5F4346475F4741502E00000099
:10D5D00073645F626C655F6366675F736574282957
:10D5E0002072657475726E65642025732077686596
:10D5F0006E20617474656D7074696E6720746F203D
:10D6000073657420424C455F4741505F4346475F16
:10D61000524F4C455F434F554E542E0073645F622A
:10D620006C655F6366675F73657428292072657433
:10D6300075726E6564202573207768656E2061744D
:10D6400074656D7074696E6720746F2073657420E3
:10D65000424C455F434F4E4E5F4346475F47415400
:10D66000542E00006E72665F626F6F746C6F61643F
:10D6700065725F77647400006E72665F6466755FE2
:10D68000626C65006E72665F6466755F666C61737E
:10D69000680000006E72665F6466755F7265715F38
:10D6A00068616E646C6572006E72665F6466755F59
:10D6B00073657474696E6773000000006E72665F54
:10D6C0006466755F73657474696E67735F737663A0
:10D6D000690000006E72665F6466755F76616C69F2
:10D6E000646174696F6E00006E72665F6466755F78
:10D6F0007665725F76616C69646174696F6E000053
:10D700006D656D5F6D6E6772000000006E72665F22
:10D710006673746F72616765000000007274745FF5
:10D720006C6F675F6261636B656E6400617070004F
:10D730006E72665F736468006E72665F7364685FC2
:10D74000626C65006E72665F7364685F736F63001E
:10D7500008200001FFFFFFFFFFFFFFFFFFFFFFFFAC
:10D7600000000000000000000000000001000000B8
:10D77000FFFFFFFF512563FCC2CAB9F3849E17A7C0
:10D78000ADFAE6BCFFFFFFFFFFFFFFFF0000000058
:10D79000FFFFFFFF96C298D84539A1F4A033EB2DC7
:10D7A000817D0377F240A463E5E6BCF847422CE1B3
:10D7B000F2D1176BF551BF376840B6CBCE5E316BF7
:10D7C0005733CE2B169E0F7C4AEBE78E9B7F1AFEBB
:10D7D000E242E34F4B60D2273E3CCE3BF6B053CC07
:10D7E000B0061D65BC86987655BDEBB3E7933AAAA3
:10D7F000D835C65A6F260700F933070015320700DF
:10D800000CD90700E82A002020010000D6370700C5
:10D810002CDA0700082C002078670000E6370700A4
:10D82000614207008541070090C607000000000024
:10D830001CD70700902B002064D6070000000404CA
:10D8400078D607000000040484D607000000040412
:10D8500094D6070000000404A8D6070000000404C2
:10D86000BCD6070000000404D4D60700000004045E
:10D87000E8D607000000040400D7070000000000FD
:10D880000CD70700000004042CD707000000040494
:10D8900030D707000000030338D707000000030358
:10D8A00044D70700000003033C2B00207830002001
:10D8B000893000208C300020F4000000A42B0020D0
:10D8C0009C2B0020A42B0020805100201800000079
:10D8D00055430700000000004585070000000000D8
:10D8E0007D850700000000008D9207000000000009
:10D8F00019940700000000005D850700000000008B
:10D9000000000000030000009D72070000000000FE
:10D91000000000000000000000000000042B0020B8
:10D92000142B002000000000000000000000000098
:10D9300000000000000000000000000000000000E7
:10D9400000000000010000000000000000000000D6
:10D95000FF00FFFF000000000000000000000000CA
:10D9600000000000000000000000000000000000B7
:10D9700001000000000000000000000000000000A6
:10D9800000E00700000000000000000000000000B0
:10D990000000000000000000000000000000000087
:10D9A0000000000000000000000000000000000077
:10D9B0000000000000000000FF000000FF03000066
:10D9C0000000000000000000000000000000000057
:10D9D00000000000000000000000000038D4070034
:10D9E000D8D3070030D40700E0D30700F0D30700F6
:10D9F000E8D30700F8D3070000D4070008D40700D5
:10DA000010D4070018D4070020D4070028D407003A
:10DA1000000000000090D0030000000000000000A3
:0CDA2000754F0700001000000000080017
:10E00000487013CC02000000010000000100000075
:10E01000000000000000000070EB00004D9A1C6D35
:10E0200001000000000000000000000000000000EF
:10E0300000000000000000000000000000000000E0
:10E0400000000000000000000000000000000000D0
:10E0500000000000000000000000000000000000C0
:10E0600000000000000000000000000000000000B0
:10E25000000000000000000000000000F6E7DFBD45
:10E2600000000000000000000000000000000000AE
:10E27000000000000000000000000000000000009E
:10E28000000000000000000000000000000000008E
:10E29000000000000000000000000000000000007E
:10E2A00000014D9A1C6D00000000000000000000FD
:10E2B000000000000000000000000000000000005E
:10E2C000000000000000000000000000000000004E
:10E2D000000000000000000000000000000000003E
:10E2E000000000000000000000000000000000002E
:10E2F000000000000000000000000000000000001E
:10E30000000000000000000000000000000000000D
:10E3100000000000000000000000000000000000FD
:04E32000000000FFFA
:10F00000487013CC02000000010000000100000065
:10F01000000000000000000070EB00004D9A1C6D25
:10F0200001000000000000000000000000000000DF
:10F0300000000000000000000000000000000000D0
:10F0400000000000000000000000000000000000C0
:10F0500000000000000000000000000000000000B0
:10F0600000000000000000000000000000000000A0
:10F25000000000000000000000000000F6E7DFBD35
:10F26000000000000000000000000000000000009E
:10F27000000000000000000000000000000000008E
:10F28000000000000000000000000000000000007E
:10F29000000000000000000000000000000000006E
:10F2A00000014D9A1C6D00000000000000000000ED
:10F2B000000000000000000000000000000000004E
:10F2C000000000000000000000000000000000003E
:10F2D000000000000000000000000000000000002E
:10F2E000000000000000000000000000000000001E
:10F2F000000000000000000000000000000000000E
:10F3000000000000000000000000000000000000FD
:10F3100000000000000000000000000000000000ED
:04F32000000000FFEA
:020000041000EA
:081014000020070000E00700C6
:00000001FF
